:1000000022C2000058C2000056C2000054C20000C4
:1000100052C2000050C200004EC200004CC200009C
:100020004AC2000048C200000C94E52E0C94CA2F6E
:100030000C94F30F40C200003EC200003CC200001E
:100040003AC2000038C2000036C2000034C20000CC
:1000500032C200000C94C12E2EC200002CC200003F
:100060002AC2000028C2000026C2000024C20000EC
:1000700022C2000020C200001EC200001CC20000FC
:100080001AC2000018C2000016C2000014C200000C
:1000900012C2000010C200000EC200000CC200001C
:1000A0000AC2000008C2000006C2000005010902E1
:1000B000A10185020901A1000509190129081500FE
:1000C0002501950875018102050109300931158165
:1000D000257F95027508810609381581257F9501D0
:1000E00075088106050C0A38021581257F95017572
:1000F000088106C0C005010980A101850319012AF4
:10010000B700150126B700950175108100C0050CD8
:100110000901A101850419012AA002150126A002E6
:10012000950175108100C00660FF0961A101096297
:10013000150026FF00952075088102096315002629
:10014000FF00952075089102C005010906A101056F
:100150000719E029E7150025019508750181029529
:1001600001750881010507190029FF150026FF0008
:100170009506750881000508190129051500250156
:10018000950575019102950175039101C00000006C
:10019000000000000000000000000000000000005F
:1001A000000000000000000000000000000000004F
:1001B000007E0F00D4FFFFFFC700000078000000A2
:1001C00000000000002A2B280000000000000000B2
:1001D000000000000000000029000000002C1E3478
:1001E00020212224342627252E362D3738271E1F7E
:1001F000202122232425263333362E37381F0405A9
:10020000060708090A0B0C0D0E0F10111213141516
:10021000161718191A1B1C1D2F3130232D350405F4
:10022000060708090A0B0C0D0E0F101112131415F6
:10023000161718191A1B1C1D2F3130354C09025B7B
:1002400000030100A03209040000010301010009BC
:100250002111010001224400070581030800010962
:100260000401000203000000092111010001222203
:100270000007058203200001070503032000010990
:100280000402000103000000092111010001227B8A
:10029000000705840320000112010002000000088D
:1002A0004350465C0100010203011C037600690013
:1002B00061006C003A0066003600340063003200D2
:1002C00062003300630000002003540068007500E2
:1002D0006D006200200054007200610063006B003A
:1002E000620061006C006C0000000E0350006C00A6
:1002F0006F006F0070007900000004030904D4004F
:10030000007ED100D300D200D500FD377A585A00C4
:100310000004E6D6B4460200210116000000742F46
:10032000E5A3E0019D00FA5D003D8889C65436C30F
:10033000174FE4E468771740EC062B597590EA1BD9
:100340009E88D5853D731290029A81140F3B0C8DC7
:10035000027F92E891B7C8CD6A298A038F8B7EB954
:1003600079E77FF380C9A7701F4EA5E2041DF2D67E
:1003700040149A79ED2C516B3D3EC5249A8FBF40B5
:100380002350F0286D98D8FF30AE076D976DBF549D
:10039000524F53BCA61B7928A634AEA70E46E1CA1D
:1003A0004CFDC54B360BD4672160ABD02A674CCDD2
:1003B000C172F58729F1DF7EC46498152C391F546A
:1003C0000CF7E3F734FC81C2C3C662278EA56CE646
:1003D0004AB6869CCD56BB06F2812A563C814579A9
:1003E000A09B665AA1C0B417C3748AA2B9C5EDFA1E
:1003F000971245E4717370624983CBF60F6459001C
:100400007C378E7E28C2113C298AD0D30067239D79
:100410001540C8701EEF0C21874CE437D9F7A44F64
:10042000E5BB00000000278AA361BB6F4D6D000192
:1004300096029E0300002D5A732DB1C467FB020083
:1004400000000004595A11241FBECFEFDAE0DEBFCE
:10045000CDBF04B603FE18C08091D5059091D60596
:10046000A091D705B091D8058730904BA740B04BED
:1004700059F41092D5051092D6051092D705109216
:10048000D805E0E0F8E3099511E0A0E0B1E0E6E38B
:10049000F9E602C005900D92A43BB107D9F725E01B
:1004A000A4EBB1E001C01D92A53DB207E1F70E94A7
:1004B00047260C941F34A4CDA4E0B0E0E2E6F2E0BD
:1004C0000C94AA312C01FB013A0129833A830B8356
:1004D0001C831701960185017401898C9A8C808197
:1004E00091814816590614F451824082D301CD906F
:1004F000DC901197C414D5041CF44D925C926201F7
:10050000A080B180C6018A199B098A309105ECF15F
:1005100063E070E00E94F5316A0D7B1D46165706B8
:100520000CF07BC0AB81BC818C91811509F470C04B
:10053000D7018D919C91DC01AA0FBB1FA20FB31FA5
:10054000CD92DC92D7018D919C9111978E319105BE
:100550000CF057C001968D939C9340815181D3013B
:100560008D919C91841B950B97FD01969595879590
:10057000840F951F91838083D3018D939C93A981D0
:10058000BA811C92AB81BC811C92AB8DBC8D8C91CD
:10059000811509F466C0D901225C3F4F80E090E0EC
:1005A0004D915D91840F951F2A173B07C9F76FE1A5
:1005B00070E00E94F5319B01D4018C91811509F402
:1005C00069C0F101A101425C5F4F80E090E0619160
:1005D0007191860F971F4E175F07C9F76FE170E0A3
:1005E0000E94F531FB01C9018E1B9F0B63E070E097
:1005F0000E94F531CB018E0F9F1F2496E2E10C94EF
:10060000C6311D921C9281E0AB8DBC8D8C93A5CF21
:1006100081E0A981BA818C93B8CF641575050CF07F
:10062000B4CFA981BA818C918115B9F0D8018D918F
:100630009C91DC01AA0FBB1FA20DB31DAD92BC9211
:10064000D8018D919C9111978E3191050CF482CF38
:100650001D921C9281E0D401D9CF81E0AB81BC8195
:10066000DACFD7016D917C91D90120E030E080E0B4
:1006700090E06115710551F4D3012D913C919CCF0F
:100680004D915D91840F951F2F5F3F4F26173707C0
:10069000BCF38FCFD8016D917C916115710581F00C
:1006A000F10140E050E080E090E0461757070CF081
:1006B00097CFA191B1918A0F9B1F4F5F5F4FF5CFED
:1006C0000190F081E02D8FCF9C019A9581159F417B
:1006D00018F5F32FF270EE27832F8170732F74704B
:1006E0006627532F5870442734FF0CC08295807FB3
:1006F000EF2B09F08062672B09F08064452B69F0CD
:1007000080680895EF2B09F08260672B09F0846000
:10071000452B19F08860089580E00895CF93DF930A
:10072000EB01D2DFFE010995DF91CF91089580930F
:10073000CB0508958093CC05089521E030E001C0F9
:10074000220F8A95EAF78091CC05822BF3CF21E026
:1007500030E0A90102C0440F551F8A95E2F7CA0193
:1007600080959091CC058923E5CF911121C08630E9
:10077000F8F491E001C0990F8A95EAF7892FE8EE25
:10078000F3E040E050E070E09191DF019B01042E26
:1007900002C0369527950A94E2F721702195292702
:1007A000282329272E934F5F5F4F4330510561F770
:1007B0000895682F892F91111CC06630D8F4E8EE97
:1007C000F3E040E050E0219130E0062E02C0369583
:1007D00027950A94E2F721703327042E01C0220FD7
:1007E0000A94EAF7822B4F5F5F4F4330510559F768
:1007F000089580E008959091CC0521E030E0F90162
:1008000001C0EE0F8A95EAF7D90102C0AA0FBB1FFB
:100810006A95E2F7EA2B01C0220F4A95EAF7892F81
:100820008E23E81303C0892F822B84CF2095822F3B
:100830008923FBCF8091960390919503981301C073
:1008400008958F5F8770FACF90911705809589235F
:1008500080931705282F2770211110C0891771F078
:100860009091CE0592FF0AC08695869586956FDF9A
:100870001092170510921905109218050895982FD7
:100880009095809114058923809314050895809193
:100890001305811531F01092130510921B0510926B
:1008A0001A050895803E9105D9F1C8F48133910568
:1008B00009F482C048F48932910509F472C08A3281
:1008C000910509F480C0089589339105E9F08238D3
:1008D0009105D1F08533910509F45EC00895843EF9
:1008E0009105D9F148F4823E910539F1833E910595
:1008F00049F181EE90E00895863E9105C9F1873E69
:10090000910509F43EC008952091CD052370211171
:1009100064C02091CE0523FF14C089E290E00895C1
:100920002091CD0520FD45C03091CE0530FF09C096
:1009300024FD24C083EE90E008952091CD0522FD92
:10094000F7CF08952091CD0522FD44C03091CE050A
:1009500030FD43C024FFF5CF11C02091CE0521FF0B
:10096000F0CF8091CD0584FD09C087EE90E0089519
:100970002091CD0523FFE5CF24FFF7CF80E090E065
:1009800008952091CD0523FD2BC03091CE0531FF78
:10099000E1CF84EE90E008952091CD0525FFD1CFE1
:1009A000BCCF2091CD0525FD1EC02091CE0523FF93
:1009B000C8CF89E390E008952091CD0526FFC1CFEF
:1009C0008AE290E008952091CD0526FFBACF81E319
:1009D00090E0089582EE90E0089580EE90E0089512
:1009E00086EE90E0089585E390E008959091CD051E
:1009F00092FF10C041E0282F2471243009F040E01C
:100A000031E0282F2871283009F030E0431711F029
:100A10002CE0822793FF10C041E0282F247124315D
:100A200009F040E031E0282F2871283109F030E04A
:100A3000431711F02CE082273091CE0530FF10C013
:100A400051E0282F2171213009F050E041E0282F9A
:100A50002871283009F040E0541711F029E082276E
:100A600031FF10C041E0282F2171213109F040E011
:100A700031E0282F2871283109F030E0431711F0B8
:100A800029E0822794FD877E08951F93CF93DF93FB
:100A900009DFEC01811522E5920708F052C08115AB
:100AA00040E5940708F0CDC0803E910520F58D3CCF
:100AB000910508F0A1C0883A910570F4853A910536
:100AC00008F097C081309105B9F10497813A9105FA
:100AD00098F1C0E0D0E030C0885A91094B97C8F730
:100AE000C85AD0E0CC0FDD1FC25CDE4F0990D88120
:100AF000C02DD46421C0811550E49507B0F4C11510
:100B000080E2D80708F0B3C0C83ED105A8F0CE01F6
:100B10009A9581159F41E8F68D2F68DF182FCE0139
:100B20009927C0DEEC01D12B07C09927BBDECC276B
:100B3000DF70C82BD92BD06ACE01DF91CF911F91E6
:100B40000895803842E59407C8F5803652E5950748
:100B500008F05BC0C03482E5D807D0F4C03292E51B
:100B6000D90708F04BC08C2F8695869520E2829F8E
:100B7000C0011124C37021E030E0A90102C0440F7C
:100B8000551FCA95E2F7EA01C82BD92BDD68D4CFEF
:100B90008C2F86958695877050E2859FC001112421
:100BA000C37021E030E0A90102C0440F551FCA956F
:100BB000E2F7EA01C82BD92BDC68BECF803C52E5B6
:100BC000950758F48F71C03AD245A0F590E0982F60
:100BD0008827EC01C46FD06AAFCF805C92458097C4
:100BE00008F077CFDC2FCC27CC27DF71C06FD06A1D
:100BF000A3CFA497D064A0CFD0659ECFCF71D0E013
:100C0000DC2FCC27C16FD06A97CF869586958770E9
:100C100020E2829FC0011124C37021E030E0A901CD
:100C200002C0440F551FCA95E2F7EA01C82BD92B21
:100C3000DA6882CFDBDEC82FD0E0DC2FCC27D06291
:100C40007BCF8F71D3DE93E0CC0FDD1F9A95E1F758
:100C5000CC27DF70282F30E084FF05C050E1859F4E
:100C6000900111243327C22BD32BD06965CF8D2F50
:100C70008F71BCDE182FCE01992714DEEC01D12B29
:100C8000DECF80E0089581152CE7920741F4209192
:100C9000820330918303232B11F480E090E00895C8
:100CA000EDE8F4E080E090E069E175E24CE355E2C4
:100CB0002EEA35E277836683518740873387228720
:100CC00097878687019670968830910599F70895E1
:100CD00010925D0510925C05ECE1F5E085818111D3
:100CE00002C014821682379685E0E435F807B1F722
:100CF0000895AC0130915F0560915E05232F62136A
:100D000001C00895822F90E0FC01EE0FFF1FEC5A06
:100D1000FA4F0190F081E02DE417F50791F467E0B8
:100D2000649FF001659FF00D1124E45EFA4F41E0ED
:100D300044832313E6CF01968370992780935F0540
:100D400008950196282F2370DACFFC018481862331
:100D500081110AC082818115B9F06823908593FFC3
:100D600005C081E061110FC080E00895282F229511
:100D70002F708F70282B962F92959F706F70962BE7
:100D800081E02913F1CF089581E00895282F35EBF4
:100D90002303C001112497FF04C080589109892FB3
:100DA000089580589F4FFBCF8091ED0380FD14C0C4
:100DB00081FD14C082FD16C08091EC03811581F085
:100DC0008E3180F420E5829FC00111246EE170E035
:100DD0000E94F531862F089584E1089588E20895F0
:100DE00088E0089580E508958091ED0380FD17C0A7
:100DF00081FD17C082FD19C08091EB03811599F028
:100E0000883298F428E0829FC001112468E270E0E3
:100E10000E94F5316115710551F0862F089562E049
:100E2000FCCF64E0FACF61E0F8CF68E0F6CF81E074
:100E30000895FA01309709F009950895E0918B0320
:100E4000F0918C03309739F00190F081E02D3097CC
:100E500011F00995089580E00895DC01E0918B037D
:100E6000F0918C03309759F086819781892B39F066
:100E700082E08C930680F781E02DCD0109950895DD
:100E8000A3E0B0E0E6E4F7E00C94BA319C01809175
:100E9000DC019091DD0182179307B1F03093DD0101
:100EA0002093DC01E0918B03F0918C03309761F08B
:100EB0000084F185E02D309739F083E089833B830E
:100EC0002A83CE01019609952396E2E00C94D6314F
:100ED000A3E0B0E0EEE6F7E00C94BA319C0180911B
:100EE000DA019091DB0182179307B1F03093DB01B7
:100EF0002093DA01E0918B03F0918C03309761F03D
:100F00000084F185E02D309739F084E089833B83BC
:100F10002A83CE01019609952396E2E00C94D631FE
:100F20009C01FC0132968FEF90E04191461751F001
:100F30008F3F19F4411101C0892F9F5F9630A9F7A7
:100F40008F3F09F40895280F311D87FD3A95F90167
:100F500062830895E8EBF1E09191891302C0DF010B
:100F60001E9291E0EE3BF907B9F70895DC01FB0111
:100F700011969C9111978181981322C012968C91A1
:100F80001297811519F0928189131AC013968C91CA
:100F90001397811519F09381891312C015968C91BE
:100FA0001597811519F0958189130AC014969C91A3
:100FB000911521F081E02481291303C080E001C054
:100FC00081E0817008958091010108952FB7F89410
:100FD0006091D6017091D7018091D8019091D9018B
:100FE0002FBF0895CF92DF92EF92FF92CF93DF93BE
:100FF000D82FC92FC0908704D0908804E09089042E
:10100000F0908A04E3DF6C197D098E099F09643F23
:1010100071408105910510F1D9DF6B017C0182E3FC
:1010200090E0A0E0B0E0C0925202D0925302E09271
:101030005402F092550280934E0290934F02A09377
:101040005002B0935102D0938504C0938604DF917F
:10105000CF91FF90EF90DF90CF90089584EF91E0D3
:10106000A0E0B0E0E0CF0895FC019B018091CC01AD
:101070009091CD018617970740F0672B29F4809156
:10108000E8008E778093E800C90140E0009741F4C2
:10109000411106C08091E80082FF2FC080E00895D2
:1010A000209184032115A9F12530A9F12091E800B0
:1010B00023FD2DC02091E80022FDECCF2091E80017
:1010C00020FFE4CF3091F3002091F200009719F057
:1010D0002830310558F041E02830310509F040E072
:1010E0002091E8002E772093E800D0CF41914093E3
:1010F000F10001972F5F3F4FE9CF80918403811565
:1011000041F0853041F08091E80083FFC3CF81E05A
:10111000089582E0089583E008958091C60187FFD5
:1011200013C08091E80082FF06C08091E8008B77B1
:101130008093E8000895809184038111F2CF08958F
:10114000809184038115D9F38091E80080FFF8CF66
:101150008091E8008E77ECCF2091E4003091E5009B
:1011600095E6A9012091EC00822F817020FF06C036
:101170008091E80080FF06C080E008952091E8009B
:1011800022FD1AC080918403811589F0853089F091
:101190008091EB0085FD0FC02091E4003091E500C7
:1011A00042175307F9F29A95E1F684E0089582E038
:1011B000089583E0089581E00895E8EDF0E08081EE
:1011C0008E7F80831092E2001092DA001092E1008C
:1011D000A0EEB0E08C9181608C9380818F778083CA
:1011E00019BCA7EDB0E08C918E7F8C9380818F7EAF
:1011F00080831092C5010895E0918B03F0918C03D8
:10120000309739F00284F385E02D309711F060E2D9
:1012100009950895982F9093E900891771F07091BE
:10122000EC002091ED005091F00021FD09C09F5F7E
:10123000973089F78093E9000895762F242F50E0A6
:101240003091EB003E7F3093EB003091ED003D7F1D
:101250003093ED003091EB0031603093EB007093F0
:10126000EC002093ED005093F0002091EE0027FD5C
:10127000DECF0895A0E0B0E0E0E4F9E00C94B431F2
:10128000C8EDD0E088818F7E8883E7EDF0E0808133
:101290008160808384E082BF81E08093C501888182
:1012A0008E7F888302EE10E0F80110821092DA003F
:1012B00081EEC82ED12CF601108288818F77888329
:1012C00088818068888388818F7D888319BC10928B
:1012D00084031092C40110924B021092C30190EE4D
:1012E000E92EF12CF70180818B7F808388818160DA
:1012F000888342E060E080E08DDFF60180818E7FB0
:101300008083F80180818160808380818860808310
:10131000F70180818E7F8083888180618883CDB74B
:10132000DEB7E8E00C94D031E091960390919503FC
:1013300029E0E91302C080E00895AE2FB0E02E9FAF
:10134000F0011124E956FC4F3181361306C030817B
:10135000381303C03581341304C0FD013196E770A2
:10136000E8CF81E0089581E08093CF054091CF05DB
:101370005091D0056091D1057091D2058FE090E039
:101380000E94753240E050E0BA0183E190E00C9495
:10139000753281E08093E00080E28093D800109263
:1013A000C9008FE097E20197F1F700C0000087E0E5
:1013B00090EBDC018093D5059093D605A093D705DB
:1013C000B093D80588E19CE00FB6F894A895809377
:1013D00060000FBE90936000FFCF0F931F93CF93D9
:1013E000DF938B01EA0190918403943051F580934F
:1013F000E9008FEF9091E80095FD06C09AE69A9576
:10140000F1F700C08A95B1F78091E80085FF19C017
:10141000A3DE811111C08091E80085FD06C0809196
:10142000E8008E778093E800F3CFF80181918F0177
:101430008093F100219779F78091E8008E7780936F
:10144000E800DF91CF911F910F910895792F6032BD
:1014500029F440E250E0682F82E0BFCF0895CF9397
:10146000DF93D82FC92F48E050E0682F792F81E013
:10147000B4DF88E0ED2FFC2FAEECB1E001900D92CF
:101480008A95E1F7DF91CF910895BC0146E050E0E5
:1014900084E0A3CFBC0143E050E084E09ECF909174
:1014A000CE0592FB222720F9281771F080FB92F9D4
:1014B0009093CE056091CD057091CE0584E090E0CB
:1014C0000E947D3282E0C0C908951F93CF93DF93BD
:1014D000962F122F632F8430B0F4911114C0463030
:1014E00090F4C42FD0E0CC0FDD1F9CE0899FC00D8D
:1014F000D11D1124CE0189960E946332612FCE0145
:101500008A960E946332DF91CF911F910895CF9305
:1015100063E472E084EF93E029DDC82F811519F0B0
:1015200084EF93E09ADC9091F50386E0E4EFF3E03A
:10153000DF01282F1D922A95E9F79093F503A3E484
:10154000B2E001900D928A95E1F781E0911101C01E
:1015500080E08C2BCF910895A4E2B0E0E2EBFAE0BA
:101560000C94AE314091F4035091F5036091F60371
:101570007091F7038091F8039091F9039FD4209321
:10158000F4033093F5034093F6035093F70360930D
:10159000F8037093F90386E0E4EFF3E0DE011796B9
:1015A00001900D928A95E1F71091F70311951A8732
:1015B00086E0FE013796DE011D9601900D928A9518
:1015C000E1F726E0FE013D96CE010196DC01019097
:1015D0000D922A95E1F726E0FC01A4EFB3E001901B
:1015E0000D922A95E1F726E0E4EFF3E0DE0117968D
:1015F00001900D922A95E1F726E0FE013796DE0173
:10160000539601900D922A95E1F726E0FE0173961C
:10161000DC0101900D922A95E1F726E0FC01A4EF90
:10162000B3E001900D922A95E1F726E0E4EFF3E0B4
:10163000DE015F9601900D922A95E1F76091F60325
:101640002091FA03D82EE92EF090F8030091F903C7
:10165000211509F46DC0062E000C770B880B990B31
:101660000E94303320E030E040E05EE30E94BC3373
:1016700020913E0230913F02409140025091410240
:101680000E9499323B014C01612F110F770B880B9F
:10169000990B0E94303320E030E040E05EE30E948E
:1016A000BC3320913A0230913B0240913C02509170
:1016B0003D020E9499325B01C82E192FB301C4016B
:1016C0000E94FD32062FB5018C2D912F0E94FD3214
:1016D000F62E602F002E000C770B880B990B0E94C2
:1016E00030339B01AC01B301C4010E949832609376
:1016F0003E0270933F0280934002909341026F2D0F
:101700000F2C000C770B880B990B0E9430339B0138
:10171000AC01B5018C2D912F0E94983260933A0252
:1017200070933B0280933C0290933D0210E060E096
:1017300069A31AA3FBA20CA386E0FE017F96DE013B
:10174000179601900D928A95E1F786E0FE01379693
:10175000AD2DBE2D01900D928A95E1F786E0ED2D1D
:10176000FE2DDE01599601900D928A95E1F786E0F3
:10177000FE017996DE01179601900D928A95E1F7A8
:1017800086E0FE013796A4EFB3E001900D928A95B2
:10179000E1F786E0EEEEF3E0DE01179601900D92A0
:1017A0008A95E1F78091F5039885892B8093F5035D
:1017B000AEDE811102C08091420210924202A496D4
:1017C000EEE00C94CA310F931F93CF93DF938430D4
:1017D00008F561111FC04630E8F4C42FD0E0CC0FEB
:1017E000DD1F2CE0829FC00DD11D1124CE018996F2
:1017F0000E944232082F10E0102F0027CE018A9657
:101800000E9442329801282BC901DF91CF911F918C
:101810000F91089580E090E0F8CF462F2091870344
:1018200030918803232B89F4703F39F4603F69F4C9
:1018300080918503909186030895711106C06630EA
:1018400020F4843010F460E0BECF80E090E0089592
:10185000A0E0B0E0EEE2FCE00C94B5317C01009138
:10186000CC058091CB05082BC3E0D0E010E0C80187
:101870000C2E02C0959587950A94E2F780FD09C069
:101880002197A8F7D12C8D2DCDB7DEB7E7E00C94CA
:10189000D131DC2EB7018C2FC0DFF7D8019781F34F
:1018A000F2CF0F931F93CF93FC0187819085009710
:1018B00089F4858100811181811581F0611571F0B4
:1018C000C801C6DFC82F682FC8010E94B503B80140
:1018D0008C2FA3DFCF911F910F910895C8010E9413
:1018E000D903C82FF4CFCF93DF93D82FC92FB0DF00
:1018F0006D2F7C2F92DFC9D8DF91CF910895FC0125
:1019000084818115A9F087819085009799F0BDD8D1
:10191000282F92959F709630B9F080F4925F9F7057
:10192000923030F4203FD1F058F481E0283E58F056
:1019300080E0089580819181D6DFEACF9A5FEFCF72
:1019400081E0243FA9F7089591E0813F09F090E0FC
:1019500081E0283E08F080E0892B089581E0089519
:10196000382F292FCB01A32FB22F873A22E09207DD
:10197000A105B10520F4875A9E4F0C94423280E0B5
:10198000089585E290E00E9442328C3789F486E225
:1019900090E00E944232833059F487E290E00E9446
:1019A000423291E08D3E09F090E0892F81700895D8
:1019B00080E0FCCFAAE0B0E0E0EEFCE00C94B431B3
:1019C000C0908203D090830381E090E090938303E2
:1019D0008093820310E08EEFE82E82E0F82E00E084
:1019E00021E030E0111104C0F701859195919C012F
:1019F000402F60E0812F69DD0F5F82E0E80EF11C6F
:101A0000063071F71F5F143031F71A8219821C8279
:101A10001B821E821D8218861F8288EC90E09A87A6
:101A2000898709E610E0FE0131967F014AE050E027
:101A3000B801C7010E948132065F1F4F093B1105A3
:101A4000A9F78AE0F70111928A95E9F74AE050E098
:101A5000B801C7010E948132065F1F4F0930F1E0D3
:101A60001F07A1F789E0F70111928A95E9F78FEF37
:101A70009FEF9E838D8387E08A874AE050E0B8011C
:101A8000C7010E948132065F1F4F0935F1E01F0731
:101A9000A1F7D0928303C09282032A96E8E00C94C7
:101AA000D031AAE0B0E0E7E5FDE00C94B431E0EE1F
:101AB000F1E080E5DF011D928A95E9F7ECE1F5E0C0
:101AC00088E3DF011D928A95E9F780EEC82E81E058
:101AD000D82E7F0109EB10E0F701D182C0824AE0E5
:101AE00050E0B801CE0101960E94323288E0FE013A
:101AF0003196D60101900D928A95E1F789859A85F4
:101B0000D70113969C938E931297BAE0CB0ED11CFB
:101B1000E7E0EE0EF11C065F1F4F0930F1E01F07F2
:101B2000D9F62A96E8E00C94D031AAE0B0E0EBE9CF
:101B3000FDE00C94B2310AE014E089E0E82EFF24C5
:101B4000F39497E0B92E2FEDC22E21E0D22EAA24D5
:101B5000A3944AE050E0B701CE0101960E943232D0
:101B6000F8013896DF018B2D1D928A95E9F789815E
:101B70009A81D80111969C938E938F8112968C93A3
:101B800012978D8113968C931397888514968C9356
:101B90001497898515968C9315978B819C81179640
:101BA0009C938E9316978A8587FD04C01E96DC92BF
:101BB000CE921D9780FF02C0F801A08681FF07C06A
:101BC000D80118969C911897926018969C9382FF62
:101BD00004C0F80190859460908783FF07C0D80106
:101BE00018969C911897986018969C9384FF04C04F
:101BF000F80190859061908785FF07C0D8011896FD
:101C00008C911897806218968C93BAE0EB0EF11CB9
:101C1000015F1F4FE9E5EE16E1E0FE0609F099CFFE
:101C20002A96EAE00C94CE31282FCB01283070F4AC
:101C30004AE0249F90011124B90167597F4F4AE07F
:101C400050E00E94323280E090E008958FEF9FEFE5
:101C50000895AAE0B0E0EFE2FEE00C94BA319C01F6
:101C600097558115914068F4BE016F5F7F4F822FB9
:101C7000DBDF892B31F489859A852A96E2E00C9482
:101C8000D63188EC90E0F9CFA0E1B0E0EAE4FEE0E4
:101C90000C94AC31FE01319680E1DF011D928A95F2
:101CA000E9F70BE210E099E5A92EBB24B39427EAEB
:101CB000422E22E0522E612C712C4F0173016201E1
:101CC000B1E14B165104610471041CF080E1C82E8F
:101CD000D12CA601B501C4010E945432AC0CBD1C2C
:101CE0000D2C000CEE08FF084C185D086E087F08EC
:101CF0000150104019F76096E0E10C94C8316FEF85
:101D000085E290E00E9463326FEF86E290E00E94ED
:101D100063326FEF87E290E00E94633260E088E216
:101D200090E00E94633246DEAFDF6CE785E290E030
:101D30000E94633263E086E290E00E9463326DEEBF
:101D400087E290E00C946332CF9324E030E043E0EC
:101D500060E080E30E940331C82F811105C00E941A
:101D600078318C2FCF91089582E08A95F1F700C0E9
:101D7000F8CFCF93C82FE8DF8115C9F08C2F0E94D0
:101D800015318FE391E00197F1F700C000000E9448
:101D90002D31C82F92E09A95F1F700C00E9478315A
:101DA00082E38A95F1F700C08C2FCF910895C0E0AF
:101DB000FBCFA2E0B0E0EFEDFEE00C94B731182FBE
:101DC000F62EC2DF082F811106C000E0802F229678
:101DD000E5E00C94D331103511F010923802106800
:101DE0001983FA8262E070E0CE0101960E944531CB
:101DF000892B59F78DE58A95F1F700000E9478311B
:101E000081E291E00197F1F700C00000DFCF60E0D0
:101E10008436910550F067E784342FE2920728F466
:101E200064E670E00E94E13161508FE0C2CF0E9411
:101E30006E308ADF811509F440C02AE62A95F1F751
:101E400000C00E9478318AE68A95F1F700C06AE501
:101E50008AE3AFDF811589F19FE728E381E09150A4
:101E600020408040E1F700C0000082E082DF83E094
:101E700080DF84E07EDF85E07CDF86E07ADF0E9421
:101E800078318FE19EE40197F1F700C000006FE028
:101E90008FE08FDF8FEC97E00197F1F700C0000033
:101EA00060E080E186DF60E081E183DF62E083E67D
:101EB00080DF80E05EDF8FE35CCF0895A8E1B0E0D3
:101EC000E4E6FFE00C94B8314B8B5C8B6D8B7E8B22
:101ED0008F8B988FFE01379686E0DF011D928A95E1
:101EE000E9F7809138028F01811108C060E080E538
:101EF00060DF811539F181E08093380225DF81159B
:101F000009F180E50E941531BDE5BA95F1F70000B1
:101F100066E070E0C8010E945E318F818770811198
:101F2000109238020E94783189859A859195819521
:101F300091099A8789878B859C85919581959109CF
:101F40009C878B8786E0FE013796DE011196019013
:101F50000D928A95E1F786E0FE013196DE011D962D
:101F600001900D928A95E1F78D8583FD05C08981E9
:101F700087FD17C01092390286E0FE017396DE01DC
:101F8000179601900D928A95E1F72F813885498542
:101F90005A856B857C8580E090E06896E4E00C943F
:101FA000D4314B815C812D813E8180913902811138
:101FB00003C081E080933902842F403851054CF0F2
:101FC0008FE78D8B822F2038310544F08FE78E8B81
:101FD000D3CF40385F4FACF780E8F3CF20383F4F86
:101FE000B4F780E8F4CF1F921FB61F9211248F938D
:101FF0009F93AF93BF9380914A02811113C0809148
:10200000D6019091D701A091D801B091D901419604
:10201000A11DB11D8093D6019093D701A093D80143
:10202000B093D901BF91AF919F918F911F901FBE27
:102030001F9018952FB7F8948091D6019091D701F1
:10204000A091D801B091D9012FBF0895CF93DF930C
:10205000C091140580911605C82B80911305811538
:10206000F1F0E8DF20911A0530911B05821B930BDC
:102070008838934110F00E944704D091130520E066
:1020800088EB91E0FC013081019631112F5F31E046
:102090008E3B9307B9F721110E944704CD2B809105
:1020A000090480958C2390910804892B8093B601B4
:1020B00048E050E06DE873E086EB91E00E941E324C
:1020C000892BB9F088E0E6EBF1E0ADE8B3E00190F0
:1020D0000D928A95E1F7E0918B03F0918C03309794
:1020E00041F00280F381E02D309719F086EB91E00A
:1020F0000995DF91CF910895811531F090911405E4
:10210000892B80931405A2CF0895811519F00E94A0
:102110003F049CCF0895811531F090911605892BCD
:102120008093160593CF0895811539F0809590918D
:10213000160589238093160589CF0895CF93DF93E1
:10214000EC014A855B856E857F850E9419079B811E
:102150009095809116058923809316058C810E94A5
:102160003F0474DF86E0FE0111928A95E9F7DF9162
:10217000CF910895CF93DF93EC018D8181FD16C03F
:1021800082608D83809116059B81892B8093160533
:10219000809114059C81892B8093140557DF488515
:1021A00059856E857F85CE010E94190710920E0514
:1021B00010920D058D8180FD02C0CE01BFDFDF9141
:1021C000CF910895962F2091CE0522FF0FC0682F42
:1021D000660F660F660F692B609317050E949D03BB
:1021E00029DF909319058093180508950C949D0399
:1021F00090911305292F2823211559F080958923C3
:1022000080931305811531F015DF80931A059093A3
:102210001B05089580E090E0F8CF0CDF2091F003DB
:102220003091F103232B211521F080937A039093B1
:102230007B032091F2033091F303232B211521F02E
:1022400080937803909379038EEE93E00C942D079E
:10225000611509F45DC0E3E3E80FE33150F4F0E009
:10226000EF5DFB4C0C9408320E94D406819580935C
:10227000F103D3CF0E94D406FACF0E94D4068195F1
:102280008093F003F6CF0E94D406FACF0E94F406A2
:102290008093F203EECF0E94F4068195F9CF0E945D
:1022A000F40681958093F303E4CF0E94F406FACFFD
:1022B000282F215D330BA90121E030E001C0220F5E
:1022C0004A95EAF79091EF03922B9093EF03409198
:1022D000F503815D21E030E0F90102C0EE0FFF1F40
:1022E0008A95E2F7CF01611509F48CC0842B8093A5
:1022F000F5030DC98091ED0381608093ED03B9CFA3
:102300008091ED038260F9CF8091ED038460F5CF79
:102310009091F003482F50E08D3C59F42091F10347
:1023200027FF0DC01092F10391110BC01092EC0326
:1023300008C08E3CB1F42091F10312169CF3911564
:10234000B1F09091F2032091F303922B911102C00E
:102350001092EB03415D51094830510508F4B7CFA5
:1023600088CF8F3C39F497FFEACF1092F003909119
:10237000F103DACF803D19F41916BCF3E0CF2091B8
:10238000F203893D29F41216D4F61092F203D7CF46
:102390008A3D19F427FFD3CFF8CF2091F3038B3D6B
:1023A00029F427FFCCCF1092F303C9CF8C3D19F449
:1023B0001216CCF3C4CF2FE2280F283080F4FA0194
:1023C000E15DF10921E030E001C0220FEA95EAF772
:1023D00020953091EF0323232093EF03B0CF20917A
:1023E000ED032E7F8D3D59F02091ED032D7F8E3D25
:1023F00031F08F3D09F0A3CF2091ED032B7F209387
:10240000ED039DCF8095842372CFCF93C82F811584
:10241000A9F08CEF8C0F813A98F4E8EBF1E08EEBA9
:1024200091E02191C21709F43DC08E179F07C9F7AB
:102430006C2F86EB91E00E94900708DECF91089503
:1024400080E28C0F883068F4C77021E030E001C072
:10245000220FCA95EAF780911405822B8093140508
:10246000ECCF8BE58C0F833038F42C2F2452330BB8
:10247000C9010E944007E2CFE8E5EC0FEB3150F4D0
:10248000F0E0EE0FFF1FEC58FE4F808191810E941B
:102490006807D4CF83E38C0F833180F661E08C2F03
:1024A000D7DECCCF8C2F0E94AA07D0DDC1CFCF932F
:1024B000DF93EC01805E9109089720F06BE870E1F2
:1024C000209711F46CE770E1CE010E948E038C2FEF
:1024D0009CDFDF91CF910895811559F19CEF980F02
:1024E000913A18F40E94AA07B1CD90E2980F983063
:1024F00050F4877091E001C0990F8A95EAF7892F0F
:102500000E943F04F1CF9BE5980F933020F480E0C8
:1025100090E00C94400798E5980F9B3120F480E000
:1025200090E00C94680793E3980F933110F460E007
:102530008FCE08951F93CF93DF93182FEB0165DFA4
:10254000209731F4812FC8DFDF91CF911F9108953B
:102550008FEC97E00197F1F700C000002197F0CFD2
:1025600060E570E0893311F060E070E0E3CFA0E057
:10257000B0E0EDEBF2E10C94B331EC018881811510
:10258000D9F0813009F03FC08981813021F48A81FE
:102590002396E6DFF3CF823021F48A81239635DF5C
:1025A000EDCF833021F48A81239696DFE7CF843004
:1025B00041F022968111E2CFCDB7DEB7E9E00C946D
:1025C000CF318A81239620E030E09AE0682F605373
:1025D000770BAB016A30710560F02115310551F3BD
:1025E000EFECF7E03197F1F700C00000215031091E
:1025F000F4CF929FB001939F700D11249A01260F82
:10260000371F8991E3CFE82FF0E0E354FE4FB490F9
:10261000282F26952695269530E0F901E355FE4FA3
:10262000E4908770F12C082E02C0F594E7940A9488
:10263000E2F7E0FAEE24FF24E0F8F901E356FE4F5A
:10264000C490D12C082E02C0D594C7940A94E2F706
:10265000C0FACC24DD24C0F8F901E357FE4F049101
:1026600010E002C0159507958A95E2F701701127D1
:10267000E114F10411F081EEC8DEC114D10411F0AF
:1026800086EEC3DE60E070E08B2D54DFC114D10410
:1026900011F086EE21DFE114F10411F081EE1CDF70
:1026A0000115110511F08CE25BDF219667CF1F93B6
:1026B000CF93DF93182FA0918304B09184041097D7
:1026C00009F449C0109286041092850410920904FE
:1026D000109208041696CD91DC911797CE019A9529
:1026E00081159F4108F4D07ED1E0C11101C0D0E036
:1026F0001996ED91FC911A97309731F01B966D91D8
:102700007C9180E00995D823D11539F08CEF8C0F9E
:10271000813A28F58C2F0E94AA071115A9F0E091A3
:102720008304F0918404808584FD0EC0809182042E
:10273000811551F0808191819C01215031092F3305
:102740003E4710F40E94F20781DC1092840410923C
:10275000830410928204DF91CF911F91089576DC5B
:102760008C2FBADEDACFCF9310921405C6E0E8EBD7
:10277000F1E0DF018C2F1D928A95E9F780E090E06F
:102780000E94400780E090E00E94680710921605C2
:102790005DDCEEEEF3E0DF011D92CA95E9F71092E1
:1027A000EC031092EB031092ED0337DDCF91089507
:1027B000DADF2FE78AE196E0215080409040E1F790
:1027C00000C0000088E19CE00FB6F894A8958093C3
:1027D00060000FBE90936000FFCFAAE2B0E0E3EF8D
:1027E000F3E10C94B93186EC91E0FC010196209163
:1027F000F100208321E08E3C9207B9F78091C70158
:10280000893009F459C0C8F4823009F4B6C0833065
:1028100009F485C0813089F18091E80083FFEAC026
:102820008091C6019091C7019A3008F0E3C0E92F6A
:10283000F0E0EC5CFB4C0C9408328A3009F48CC05C
:102840008B3051F78091C601813231F78091CA01F6
:102850009091CB01892B01F78091E800877F8093CD
:10286000E8000E948D0881E09091C801911101C09B
:1028700080E08093020177DFCFCF8091C601813A5B
:1028800059F68091E800877F8093E8008091CA0123
:102890009091CB01892B61F060E080E090E070E0E6
:1028A0000E9434088091E8008B778093E800B4CFD1
:1028B00068E08EEC91E0F3CF8091C601813209F09F
:1028C000ABCF8091CA019091CB018D7F892B09F00C
:1028D000A3CF8091E800877F8093E8008091E80093
:1028E00082FF18C09091F3008091F200029731F4BA
:1028F0008091F100813011F0863021F48091F10057
:10290000809301018091E8008B778093E8000E941A
:102910008D0882CF809184038111E0CF7DCF80919B
:10292000C601813A09F078CF8091CA019091CB011C
:10293000892B09F071CF8091E800877F8093E800B0
:102940008091E80080FFFCCF809102018093F1002C
:102950008091E8008E77D9CF8091C601813209F04D
:102960005BCF8091E800877F8093E8000E948D080C
:102970008091C901809300014FCF8091C601813AB7
:1029800009F04ACF8091E800877F8093E80080912A
:10299000E80080FFFCCF80910001D8CF803889F01B
:1029A000823841F58091CA018F70873018F5809385
:1029B000E9008091EB0085FB882780F91092E900FF
:1029C00006C080914B02880F9091C301892B909192
:1029D000E800977F9093E8008093F1001092F10057
:1029E0008091E8008E7723C0811116C08091C801C4
:1029F000813011F18091E80083FF0AC08091E800E6
:102A0000877F8093E8008091EB0080628093EB00E9
:102A1000AA96E3E00C94D531823061F78091C80129
:102A2000811589F01092E9008091E800877F8093FA
:102A3000E8000E948D08DECF81E0933009F080E04D
:102A400080934B02EFCF8091CA018F702FEF280F38
:102A5000263080F68093E9002091EB0020FFE2CF42
:102A6000933031F48091EB0080628093EB00DACFF9
:102A70009091EB0090619093EB0021E030E0A90190
:102A800002C0440F551F8A95E2F74093EA00109266
:102A9000EA008091EB008860E8CF8111ABCF109104
:102AA000C8011F778091E3008078812B8093E30039
:102AB0008091E800877F8093E8000E948D088091D4
:102AC000E80080FFFCCF8091E30080688093E30002
:102AD00083E0111101C082E0809384038BCF805882
:102AE000823008F087CF8091C8019091C9018C3D58
:102AF00053E0950799F583E08A838AE289834FB78B
:102B0000F894DE01139620E03EE051E2E32FF0E07E
:102B100050935700849120FF03C082958F703F5FD0
:102B20008F708A30C8F0895C90E08D939D932F5F01
:102B3000243161F74FBF8091E800877F8093E800E0
:102B40006AE270E0CE0101960E9434088091E800AC
:102B50008B778093E8004ECF805DE6CF292F332717
:102B60002330310509F44EC078F52130310509F4E0
:102B700088C08BE590E0EDE3F2E02230310509F00A
:102B800039CF2091E800277F2093E8002091CC01E5
:102B90003091CD018217930708F49C0140E0211584
:102BA000310509F073C0411171C08091E80082FDC8
:102BB000CDCF80918403811549F2853039F280911F
:102BC000E80083FFF2CFC2CF8091CA019091CB0180
:102BD0002132310509F446C02232310509F00ACF0D
:102BE0008330910508F006CFFC01EE0FFF1FE45D76
:102BF000FE4F0190F081E02D875D9E4FDC018C91AE
:102C000090E010C09C013327823021F12330310540
:102C100068F4232BB9F4EAEFF2E0E4918E2F90E010
:102C2000EAEFF2E0009709F4E5CEABCF23303105AF
:102C300009F0E0CEEAEAF2E0E4918E2F90E0EAEAD1
:102C4000F2E0F0CFEAEEF2E0E4918E2F90E0EAEECF
:102C5000F2E0E8CFE8ECF2E0E4918E2F90E0E8ECCF
:102C6000F2E0E0CF8330910508F0C4CEFC01EE0F16
:102C7000FF1FEE5CFE4F0190F081E02D89E090E0B7
:102C800080CF82E190E0E8E9F2E07BCF809184039D
:102C9000811509F45BCF853009F458CF8091E800A5
:102CA00083FD54CF8091E80082FD7FCF8091E800C2
:102CB00080FF75CF9091F3008091F20021153105CE
:102CC00019F08830910550F041E0089709F040E094
:102CD0008091E8008E778093E80061CF4491409323
:102CE000F1003196215031090196E8CF803809F082
:102CF00081CE8091E800877F8093E8008091C401B5
:102D00008093F1006DCE811175CE1091C801123003
:102D100008F070CE8091E800877F8093E8001093E0
:102D2000C4010E948D081115F9F084E0809384039A
:102D300042E061EC81E00E940A0942E261EC84E039
:102D40000E940A0942E261EC82E00E940A0942E222
:102D500060EC83E00E940A0980918403843051F47E
:102D600082E08093030146CE8091E30087FDDDCFB2
:102D700081E0DCCF81E0F5CFA0E0B0E0E2ECF6E16D
:102D80000C94B531162FD72FC42FD22E811599F060
:102D9000409311054FD99093C2018093C101C77030
:102DA00081E001C0880FCA95EAF7A6D9CDB7DEB792
:102DB000E7E00C94D13190911105491333C0E090B4
:102DC000C101F090C20136D99C012E193F09790149
:102DD000812F9D2F0E94290EE816F90618F5D0E2E2
:102DE000DD0DCD1591F0C77011E0812F01C0880F66
:102DF000CA95EAF78AD9D83040F48D2D877001C082
:102E0000110F8A95EAF7812F77D9802FA9DBD83067
:102E100068F62D2D277081E001C0880F2A95EAF70A
:102E200074D9C4CFC77081E001C0880FCA95EAF792
:102E3000F7CFACE0B0E0EFE1F7E10C94AB317C010F
:102E4000DC0114968C91811509F4E2C161E0C7019F
:102E50000E94510C8C01F7018581811529F1809127
:102E60000D0590910E050097F9F008171907E1F08C
:102E7000FC01FF27887F9927892B09F0A7C0A4E0D0
:102E8000EE0FFF1FAA95E1F7E357FB4F85818460A2
:102E9000858311830083CF016DD91092160561E0FF
:102EA000C7010E94510C8C01D7018C91813069F4CB
:102EB00011968C91811109C0BDD89093FD03809328
:102EC000FC03F70185818093FB03D70115968C9154
:102ED0000115BEE71B0709F07CC0811509F180913F
:102EE000CF0590E0019665E070E00E94E1318093AB
:102EF000CF054091CF055091D0056091D1057091DB
:102F0000D2058FE090E00E947532E091CF05F0E0AD
:102F1000EE0FFF1FE655FE4F808191810E94070F43
:102F2000D70115968C91811163C06801A7E5DA1A63
:102F3000C114B1E0DB0668F56EEF73E08C2D0E94E2
:102F4000140E892B31F5C60154E0880F991F5A954C
:102F5000E1F7FC01E357FB4F2281213009F02FC13B
:102F60002091FE033091FF03232B99F02091000460
:102F700030910104232B69F0209102043091030465
:102F80004091040450910504242B352B232B09F484
:102F900020C1F7013580311409F43EC10E35FCE73C
:102FA0001F0709F421C10F352CE7120751F00D3529
:102FB0003CE7130709F030C180911001811509F435
:102FC00013C11092100180E072DB11C1E0E0F0E06B
:102FD0005DCF0130EEE71E0709F0A2CF811509F49D
:102FE0009FCF8091FA0391E089278093FA0398CFCD
:102FF000C80197578038910560F6003108F0F7C096
:1030000066EA72E080E090E00E94B00C8111EFC0AF
:10301000812C912C5401011146C004E09E012F5FC8
:103020003F4F6901D601E02F1D92EA95E9F724018F
:103030003501FFEF4F1A5F0A6F0A7F0AC501B4011D
:103040000E94B00C8983811509F4D1C0813009F048
:10305000B3C0A50194012E5F3F4F4F4F5F4F2D83AB
:103060003E834F835887C301B2010E94B00C182FD2
:103070008A83811509F4BBC08FEF810F833078F507
:103080006D817E818F8198850E94B00C8B83811524
:1030900011F0C6016CDA2401350133E0430E511CF6
:1030A000611C711C19C0B7EA8B16B2E09B06A10423
:1030B000B10409F49CC0C501B4010E94B00CEFEF4B
:1030C0008E1A9E0AAE0ABE0A8111EDCF0150A3CF1F
:1030D0004D805E806F80788453014201A3CF8BEFD7
:1030E000810F8330A0F52401350143E0440E511CCB
:1030F000611C711C6D817E818F8198850E94B00C4E
:103100008B83811549F3C301B2010E94B00C8C83FB
:10311000811108C02401350154E0450E511C611C89
:10312000711CDACF8B819C818130AFEF9A0710F050
:10313000982F8827163029F0173031F00E940E257D
:10314000E9CF0E94BB24E6CF0E94DC24E3CF1430F9
:1031500009F0BECF6D817E818F8198850E94B00C71
:10316000182F24013501B4E04B0E511C611C711C59
:10317000C501B4016D5F7F4F8F4F9F4F0E94B00C10
:103180001115A9F1811599F18150990B4FEF489FC5
:103190009001499F300D1124E12FE150FF0B2E0FBC
:1031A0003F1F2150310908F497CF8FEC97E001972A
:1031B000F1F700C00000F5CFC601D9D98DCF22307C
:1031C00009F0E7CE2091020430910304232B09F487
:1031D000E0CEFC01EE56FB4F20812E7F20838357EB
:1031E0009B4F0E94BA10D5CE81E080931001809150
:1031F00017058770811561F0D70115968C9181159F
:1032000039F08091CE0582FF03C082E00E94240441
:103210002C96E1E10C94C73180911001811168C0B6
:10322000C80197558115914008F0FDC05801F8EF8D
:10323000AF22BB24A114B104D1F6F801FF2734E07A
:10324000EE0FFF1F3A95E1F79F0123573B4F6901AE
:10325000D70115968C91EE56FB4F908180FB90F92B
:103260009083811509F4D8C10E941A10909310051B
:1032700080930F05F60182818F5F8283809116050E
:1032800090911405892B8383809113058483468153
:10329000578166857785C6010E941907D601159664
:1032A0008C9181FF5801B0920E05A0920D05D701B7
:1032B00015968C91811509F4A7C5109211059801F6
:1032C00030572332310508F088C584E090E00E9431
:1032D0004F329093CE058093CD05F801E150F04731
:1032E000E232F10508F0E0C1E25CFB4C0C940832DC
:1032F000380150EE651A710850901505809114053B
:10330000582A80911305582A88E06816710408F03D
:103310005EC098012770332781E090E001C0880FDC
:103320002A95EAF7311409F44FC0582AD7018D9134
:103330009C910E94D90321E030E0F90102C0EE0F18
:10334000FF1F8A95E2F7FE83ED832091830430917D
:1033500084043A87298740918B0450918C045C87C0
:103360004B874AE0C42E44E0D42EA12CB12C51103E
:1033700005C0D60112968C9181111BC0F601838184
:1033800090E02D813E8182239323892B91F08085CB
:10339000982F9770911101C087E038E0631671048F
:1033A00008F065C0311409F45EC086958170811102
:1033B00063C09FEFA91AB90AAFE0CA0ED11CB8E0EA
:1033C000AB16B104A1F61CC080955822AFCF3110C6
:1033D00037C080918B0490918C040817190781F4F1
:1033E00010928C0410928B0410928704109288041F
:1033F0001092890410928A04109286041092850417
:103400008091830490918404009709F409CFE8E047
:103410006E16710408F0EBC0652D0E94A50681119F
:1034200002C081E044D9F7018581F801E851FC47E9
:10343000E730F10508F03BCFE05AFB4C0C94083222
:1034400010938C0400938B040E94E607609387041A
:10345000709388048093890490938A041092860460
:103460001092850463CF82FB882780F9A0CF3114A6
:1034700009F49FCF80FF9DCFD6018D909C900815B9
:10348000190519F4311409F494CFE985FA85EC157E
:10349000FD0509F48ECFD6011D96ED91FC91309774
:1034A00021F08081811509F484CF652DC6010E9429
:1034B000A506811509F47DCF81E00815190509F0ED
:1034C00080E0482E43208114910441F0411006C051
:1034D000EB85FC858E169F0609F06BCF80E0E7D860
:1034E000D0928404C092830481E0809382048FE0B0
:1034F0008A9DF0018B9DF00D1124E65FFB4F8581C5
:103500008093090441100EC08114910459F0808108
:1035100091819C0124503109213A310508F049C0BC
:103520000E94AA078FE08A9DF0018B9DF00D112467
:10353000E65FFB4FC680D780C6019A9581159F41F3
:1035400010F420EED22299249394C60101978F3370
:103550009E4708F0912C8FE08A9DD0018B9DB00D85
:103560001124A65FBB4F1996ED91FC911A973097E5
:1035700031F01B966D917C9181E009959822911410
:10358000A9F08FE08A9DF0018B9DF00D1124E65F7C
:10359000FB4F868197810E94640380930804C601D3
:1035A00048E06416710440F40E94F2070E9426105D
:1035B0000CC00E946C12B6CF0497813A910558F462
:1035C0006C2D86EB91E00E949007411409F428CEFF
:1035D0000E9426100CCE0E9426108FE19EE40197D7
:1035E000F1F700C000008C2D0E940512EECFDC0127
:1035F0002D913C910217130739F4311008C0109235
:10360000820480E054D80CCE311409F409CEFC01B8
:10361000808585FD05CEF5CFF90144855585668504
:103620007785C9010E941907D60115968C9181FFF3
:103630003ECEC6010E949E1080910D0590910E0510
:103640000817190709F033CE10920E0510920D05D8
:103650002ECE06E221EE41EE6AE17CE78DDBC7CD9E
:1036600007E225EE45EE6BE17CE7F8CF06E221EEBE
:1036700040EE68E17CE7F2CF07E225EE44EE69E137
:103680007CE7ECCF06E221EE42EE6CE17CE7E6CF90
:1036900007E225EE46EE6DE17CE7E0CF08E221E0AF
:1036A00045EE6EE17CE7DACF8091CD0581608093B5
:1036B000CD056091CD057091CE0584E090E00E942B
:1036C0007D3251D894CD8091CE0588608093CE050F
:1036D000F0CF8091CD058260EACF8091CD058460E6
:1036E000E6CF8091CD058860E2CF8091CE058160E4
:1036F000EDCF8091CE058260E9CF8091CD058061CC
:10370000D6CF8091CD058062D2CF8091CD058064E7
:10371000CECF29D88091CD058068C9CF8091CD05C5
:103720008C60C5CF8091CE058360D0CF8091CD05D0
:103730008E7FBDCF8091CE05877FC8CF8091CD058C
:103740008D7FB5CF8091CD058B7FB1CF8091CD0599
:10375000877FADCF8091CE058E7FB8CF8091CE058B
:103760008D7FB4CF8091CD058F7EA1CF8091CD0587
:103770008F7D9DCF8091CD058F7B99CF0E94B31314
:103780008091CD058F7793CF8091CD05837F8FCFAB
:103790008091CE058C7F9ACF8091CD05992782FFAD
:1037A000939590FB82F990FB83F981CF8091CE05B0
:1037B000982F909590FB80F990FB81F987CF90919D
:1037C000CD05892F8F7B96FF806471CF0E94B31344
:1037D0009091CD05892F97FB87F9805868CF61E0DC
:1037E0008EE090E00E94633264CF60E0F9CF909168
:1037F000CD05892F8F7E94FF806159CF9091CD05A3
:10380000892F8E7F90FF816052CF9091CE05892FB6
:10381000877F93FF88605ACF89E201C30737BCE7EF
:103820001B07F9F00837ECE71E0751F19801205EFD
:1038300032452032310550F581113FC00F7181E0D2
:1038400090E09C0102C0220F331F0A95E2F7890124
:10385000622F83E090E00E946332802F0E949703E2
:10386000C6CC811549F081E00E949D0343E062E0EF
:1038700081E00E94FB03BBCC81E00E94A703F6CF4E
:10388000811511F082E0F0CF82E0F7CF8115A9F029
:103890000A353CE7130709F476C008F04EC0013042
:1038A0005CE7150709F46DC003308CE7180709F4CD
:1038B00062C001151C4709F451C0F701878190854A
:1038C000009709F464C00E9445058C01F701B5809A
:1038D000A680A2942FE0A2228091170587708115FF
:1038E00001F1CB2CB114F1F0812F807F803461F095
:1038F00080E2800F8830A8F0812F807E803221F412
:10390000023078F0A11469F08091CE0582FF09C0E1
:1039100082E00E942404809117058770CC24C39410
:103920008111C12CE12FE295EF70103C08F0A5C089
:10393000F0E0E959FB4C0C9408320B35ACE71A0760
:1039400021F18091CE05002482FF0394802D0C3557
:103950001C4709F0B2CF0E944F0AAFCF0E94B313A9
:10396000EFE7FAE126E0E150F0402040E1F700C047
:1039700000000E94C9096FEF7FEF80E090E00E9495
:103980007D320E94D81381E0E6CF80E0E4CF8581CC
:10399000C080D180811569F0C6010E94280C182FC3
:1039A000682FC6010E94B503B601812F0E940D0C3D
:1039B0008ACFC6010E94D903182FF6CFF12FFF70CE
:1039C000DF2E103118F0D29490EFD922B114B9F053
:1039D000D11469F080E2800F883010F0011109C025
:1039E000809114058D29809314050E942610802F44
:1039F00042C0809116058D2980931605F6CF802F41
:103A00000E946C12D114C9F180E2800F883010F04E
:103A1000011104C08D2D0E943F0406C0D0948091F6
:103A200016058D21809316050E94261026C0212F91
:103A30002F70D22E107F103219F0D29480EFD8223E
:103A4000011549F0013009F484C0B11409F490C0A3
:103A5000A114B1F1CCCF8091CE0582FD2DC0B1145F
:103A600029F1D11439F0809114058D298093140522
:103A70000E94261080E00E940512C11409F4D8C0EB
:103A80008091170580FDD4C0D70115961C928695AC
:103A9000869586950E949D03C701CBD98091170515
:103AA0008695869586950E94A703C2C080E00E94F5
:103AB0006C12D11411F3AECFB11469F1A11004C08E
:103AC0008D2D0E947C10D9CF31E0A31210C010912F
:103AD00013058D2D8123D81681F20E941A10909320
:103AE0001B0580931A051D2910931305C6CF45E0C9
:103AF000A412C3CF8D2D0E947C108D2D0E94F81032
:103B0000809115059D2D9823D91609F4B6CF8D29DE
:103B100080931505B2CFA11012C08D2D0E94851083
:103B20008D2D0E94F810809115059D2D98239115DB
:103B300009F4A3CFD094D822D09215059ECF51E09E
:103B4000A5129BCF809114058D21811509F495CF85
:103B5000E4CFB11429F086E0A81608F08ECFB0CFDC
:103B600095E0A91608F089CF8D2D0E94851085CF8C
:103B7000A114D1F3093349F4AFEFB3EFE1E0A15061
:103B8000B040E040E1F700C00000802F0E946C12BE
:103B900074CF812F869586958370811561F0813071
:103BA00009F06BCFC8019370B11002C080E090E0C3
:103BB0000E94680762CFC8019370B11002C080E014
:103BC00090E00E94400759CF6B2D802F0E94281152
:103BD00054CF812F8370811138C0B11027C0402F7E
:103BE000429546954770440F440F802F8F70042EE6
:103BF00001C0880F0A94EAF7202F207104FF07C044
:103C00002FE030E001C0220F4A95EAF72095169583
:103C1000169513701230A1F0133081F03091CB055E
:103C2000113059F0822B83230E9497030E941E07B4
:103C300060E0C7010E94510CEBCA832B822BF4CFAA
:103C4000822B9091CB058927EFCFB11451F110FF52
:103C5000EDCF402F429546954770440F440F802F7B
:103C60008F70042E01C0880F0A94EAF7202F20716C
:103C700004FF07C02FE030E001C0220F4A95EAF7A9
:103C80002095169516951370123089F0133069F04F
:103C90003091CC05113041F0822B83230E949A038E
:103CA000C5CF823018F2D5CF832B822BF7CF822B52
:103CB0009091CC058927F2CF1F70B11439F0812F74
:103CC0000E949D03802F0E947C10B0CF802F0E9405
:103CD0008510812F0E94A703A9CF023F71F170F4D4
:103CE000003FC9F0013F91F0B11409F465C0A1147F
:103CF00009F45FC0802F0E94051298CF033F21F185
:103D0000043F91F78091CE0582FD2AC0812F8F71EB
:103D1000B11401F316C0B11469F0F5E0AF1608F064
:103D200085CF1F7181E090E0012E01C0880F0A94B9
:103D3000EAF7BECF26E0A216F2CF812F8F71B11025
:103D4000C9CF0E949D0372CF80E0B11409F4A6CFC1
:103D50001F7181E0012E01C0880F0A94EAF79ECFFF
:103D6000B114C1F0809117058770843049F4109226
:103D700017051092190510921805812F8F71AACF7F
:103D800035E063E0A31608F051CF812F8F710E94B8
:103D9000E2104CCF45E0A41640F0109217051092A7
:103DA00019051092180564E0F0CF81E00E94240408
:103DB0003DCF812F8F71C5CFA114F9F2093349F49A
:103DC0005FEF83EF91E0515080409040E1F700C0F9
:103DD0000000802F0E946C1229CF0631BCE71B0720
:103DE00009F01CCD809114058A7A91E0811101C0FF
:103DF00090E09093120565E3811101C069E286EBC2
:103E000091E00E949007E4CB0631ECE71E0709F031
:103E100005CD80911205811509F4FECC85E30E9441
:103E2000AA07D6CBA0E0B0E0E8E1FFE10C94B53101
:103E30008091E503803108F049C08091E403811549
:103E400009F444C0C091960389E0D82E809195036F
:103E50008C17E1F1EC2EF12CDC9EE0011124FE0127
:103E6000E956FC4F84818115B1F191818091E00385
:103E7000981331C090818091DF0398132CC0858105
:103E8000811129C0028113818091E1039091E203A5
:103E9000081B190B60E08FED93E00E94510C0E940B
:103EA000290E08171907B8F48091E5038F70806117
:103EB0008093E503C356DC4F88818F7080618883CF
:103EC0008FED93E00E9419170E941A04CDB7DEB758
:103ED000E7E00C94D131E7012196C770B7CFAFE08E
:103EE000B0E0E5E7FFE10C94AD318C0186E0F8012C
:103EF000DE011A9601900D928A95E1F7F801F5809E
:103F0000E4808FED882E83E0982E8091E303811169
:103F100017C0E11491F0F11409F480C1C8010E94A6
:103F20007F0C811509F47AC189E0F801AFEDB3E0A7
:103F300001900D928A95E1F775DFFF24F3946AC032
:103F4000A280B380D090E4038091E1039091E203DA
:103F50003501681A790AD11409F411C1C080518061
:103F600060E08FED93E00E94510C0E94290E6816CC
:103F7000790608F0B6C0E11401F38091E003F8017E
:103F80009181E090E503F0E1EF1608F064C098132A
:103F900020C09091DF03F801808198131AC020910E
:103FA000E6033091E703878190852817390789F464
:103FB000F1104BC08E2D8F7080618093E5038FEDE3
:103FC00093E00E9419178091E503F8018683F12C94
:103FD00021C0F1103AC040E0652D8C2D0E9494095B
:103FE00040E0652D8C2D0E949409F82E8111EFCFB1
:103FF0008A859B850E94730C292F22952F709034FF
:1040000070F49F702230A0F09115B1F0F801968104
:10401000903190F48F2D2F96EFE00C94C9312A5FE8
:104020002F70223068F0C8010E941917FD2CF2CFC2
:10403000911511F0811571F3805E883058F3F3CF3C
:10404000803F40F3815F8330F9CF8091E503816049
:104050008093E503BCCF98131EC09091DF03F80155
:104060008081981318C02091E6033091E70387817F
:1040700090852817390779F4F1100DC0E682C80140
:104080000E94191789E0F801AFEDB3E001900D929D
:104090008A95E1F752CFC8010E947F0C811509F47F
:1040A000BDC0F11409F4BAC08091E503803208F470
:1040B0003BCF8091DF039091E0039A838983BC8298
:1040C000AB828091E3038D831E82EF828091E603B1
:1040D0009091E70399878887CE0101960E9419176E
:1040E00023CFD090E503F0E1DF1650F48FED93E09D
:1040F0000E94191789E0F40111928A95E9F767CFB8
:10410000E11409F41ACF9091E003F801818198132A
:104110001AC09091DF038081981315C02091E603A7
:104120003091E703878190852817390761F4F110F2
:104130000AC0D682C8010E94191789E0F4011192C1
:104140008A95E9F7FACEC8010E947F0C811509F41F
:1041500065C0F11409F462C08091E503803208F46F
:10416000E3CE8091DF039091E0039A838983BC8240
:10417000AB828091E3038D831E82DF82A7CF60E054
:104180008FED93E00E94510C0E94290E681679066B
:1041900008F0B0CFE11409F4D0CEF11409F43EC018
:1041A0009091E003F801818198132EC09091DF0374
:1041B0008081981329C02091E6033091E70387811D
:1041C00090852817390701F58091E1039091E2036A
:1041D000A81AB90AF8ECAF16B10408F053CF8091D1
:1041E000E50380FD4FCF803108F44CCFF801868382
:1041F000982F907F903F09F442CF982F907F905F47
:104200008F70892B86833BCFC8010E947F0C811160
:104210008BCE8091E50381608093E503C8010E9405
:1042200019178BCEA2E1B0E0E8E1F1E20C94B831CD
:104230000A871B872C873D874E875F87688B798B22
:104240008A8BCE010A964BDE811128C020919503FE
:104250003091960389E0FE013A96DE0111960190B5
:104260000D928A95E1F78E858115C1F0822F90E03D
:1042700001968770992738171906D9F099E0929F0F
:10428000D0011124A956BC4FFE01319601900D9228
:104290009A95E1F7809395030E941A0419E08091A2
:1042A000960390919503891312C06296E4E00C94F2
:1042B000D4310E94B313109295031092960389E0B3
:1042C000EFEDF3E0DF011D928A95E9F7E7CF189F44
:1042D000C001112489569C4F02DE811531F3809173
:1042E000960390E001968770992780939603D7CF25
:1042F000EF92FF920F931F93CF93DF938091C805A6
:10430000E091DE01CDE0811130C0CDB7DEB7E6E04F
:104310000C94D231D1E0DE0FD093DE01EE2EF12CE1
:10432000CE9FF0011124E05AFA4F84818115E1F00B
:1043300087819085892B21F481859285019651F49E
:104340000081118122813381448155816681778189
:10435000808568DFCE9DF001CF9DF00D1124E05ADD
:10436000FA4F148210921605ED2F8091C805E817B8
:1043700088F21092C8051092DE01C7CFA4E0B0E029
:10438000E4ECF1E20C94AB3120915F05298397E0D6
:10439000992E01E010E02DE0322E34E0532E8824D7
:1043A000839480915E059981891307C0A1DF0E94E3
:1043B00068062496E1E10C94C7319981892F90E039
:1043C0009C838B83FC01EE0FFF1FEC5AFA4F808118
:1043D0009181989ED001999EB00D1124FD01E45E5B
:1043E000FA4FFA83E983248121115BC06090C805EC
:1043F000E0E6F5E060E070E0712C661508F04FC073
:10440000A384B484A981BA81CD90DC902FEF3FEFD3
:10441000412C442D50E07601E40CF11CE40CF11C1D
:10442000D701ED90FC90E114F10439F0AE14BF0413
:1044300009F0A90143949A01ECCF2F3F3207D1F143
:10444000D80102C0AA0FBB1F2A95E2F77A2A980169
:10445000042C02C0220F331F0A94E2F7A901415035
:1044600051097416150629F5369EF001379EF00D98
:104470001124E05AFA4F989ED001999EB00D112454
:10448000A45EBA4F12962D913C91139730872783E3
:104490005482108211829287818715968C920E9495
:1044A00079068B819C8101969A83898383708983A5
:1044B00078CF14826F5F7F4F3D969FCF1092CA05D1
:1044C0001092C9051092110180915E0580935F05DD
:1044D0000E9468060DCFACE1B0E0E1E7F2E20C9497
:1044E000AA314B8B5C8B6D8B7E8B8F8BB92E988F0B
:1044F000A92E911110921605188A198A1A8A86E037
:10450000FE017396DE011A9601900D928A95E1F7ED
:104510005F888091CE0582FF1FC00E941A102091F3
:10452000180530911905821B930B8838934138F098
:104530008091170582FD03C082E00E9424040E943E
:104540001A1020911A0530911B05821B930B883895
:10455000934110F00E9447045114D9F05E86BF8643
:1045600061E0CE010A960E94510C61E0CE010A96EC
:104570000E94510C61E0CE010A960E94510C4C0140
:1045800080356CE7960791F4A11419F181E08093CE
:1045900011015E86BF860A851B852C853D85452DCC
:1045A0005B2D688979898A893DDECDC081359C473C
:1045B00021F4A11471F082DFECCF82E588168CE73C
:1045C000980639F4A11429F0809111018111F3CFDB
:1045D000DDCF4CE1E42E45E0F42E412C612C712C12
:1045E000D7016D917C91CC24CA94DD24DA9480E0CB
:1045F000282F30E0FB01E80FF11DE80FF11D40818D
:1046000051814115510539F08416950609F096013E
:104610008F5F6901EDCF10E0BFEFCB16DB0609F429
:104620004EC0F701448110911101411110E0D701F2
:1046300015963C90159716969C911697A11409F41F
:1046400005C1111509F402C1311017C021E030E095
:104650000C2C01C0220F0A94EAF7922B16969C9319
:1046600020915C0530915D052233310530F422E361
:1046700030E030935D0520935C05E1E0F0E002C09E
:10468000EE0FFF1F8A95E2F7CF010197D70116962B
:104690002C912817190699F4C090C905D090CA0525
:1046A000C114D10409F453C00E941A108C199D0939
:1046B000C39708F44CC081E0F701848311E0412ADC
:1046C000BFEF6B1A7B0AE7E0EE0EF11CF8E06F1605
:1046D000710409F085CFA11409F417C1411409F43C
:1046E00014C10E941A109093CA058093C905809145
:1046F000C805883040F591E0980F9093C80599E07F
:10470000FE013A96DE01119601900D929A95E1F71D
:104710005D82BE822DE0829FC0011124805A9A4F93
:1047200029E0FE013196DC0101900D922A95E1F716
:104730002FEF3FEFDC011A963C932E9319971C96AE
:104740009C928E921B976C96E2E10C94C63120915C
:104750005F0580915E05922FE0E0F0E001E0281710
:1047600009F448C0422F50E0FA01EE0FFF1FEC5A47
:10477000FA4F2080318037E0329DF001339DF00DFB
:104780001124E45EFA4F608171817C8F6B8FB0E001
:1047900030E0A0E0EB8DFC8DEA0FF11DEA0FF11D7A
:1047A000C080D180C114D104E1F0F7010190F08103
:1047B000E02DFA8FE98F30E007C0E1E0C616D7069A
:1047C00009F0E0E0BE2B3F5FE98DFA8DE30FF11DAC
:1047D000E30FF11D608171816115710571F7AF5FA4
:1047E000D9CFB11581F13A17C8F4E1E0D701149699
:1047F000EC93F70190935F05EE15FF0509F45FCF89
:1048000090E0FC01EE0FFF1FEC5AFA4F71826082BC
:1048100001968370992780935E0551CF37E0329DD2
:10482000F001339DF00D1124E45EFA4F0483EE1580
:10483000FF05F9F2291302C09F5F93709A012F5F61
:104840003F4F23708CCFE0E0F0E0F8CF292F30E02D
:10485000311024C061E070E002C0660F771F8A95B6
:10486000E2F7CB0101972817390791F010E0E1E05A
:10487000F0E002C0EE0FFF1FCA94E2F76F01C09490
:10488000D70116968C9116978C2116968C9317CF7C
:10489000411569F3C3010E947906E8CFA9010C2CE8
:1048A00002C0559547950A94E2F7C9010197822302
:1048B0009323892B39F540FF25C0D70112968D919E
:1048C0009C91892BD1F087E0FE013196DF011D928A
:1048D0008A95E9F70E941A109C018B839C8384E0DF
:1048E0008D83F70192818381792F98878987098148
:1048F0001A8144E05E816F8195DCD70115961C9288
:10490000132DB5CF142F1170B2CF90915F05809108
:104910005E05981731F032DDB1E04B1609F413CF84
:1049200038CEE6DC1092CA051092C9050E946806CE
:10493000F3CFA6E0B0E0EFE9F4E20C94B8310E94C6
:104940001A108C018091890390918A038017910736
:1049500071F019821A820E941A10BC0149815A8191
:1049600080E090E0B8DD10938A03009389032696D7
:10497000E4E00C94D431A6E0B0E0E1ECF4E20C9475
:10498000BA319093860380938503811520E29207C4
:1049900030F40E9457122696E2E00C94D63180EF54
:1049A00089838A830E941A108160BC0149815A81DF
:1049B00081E091E090DDEFCFA6E0B0E0E2EEF4E23E
:1049C0000C94B8318C019093860380938503011574
:1049D00080E21807B0F4802F0E946C12C801805E3C
:1049E0009109089728F064E970E10115110511F4A7
:1049F00065E870E1C8010E948E032696E4E00C94FD
:104A0000D43180EF89838A830E941A108160BC01AF
:104A100049815A8181E090E05EDDEFCFCF93DF9353
:104A2000D82FC92FA8DF8D2F9C2FC6DFDF91CF9104
:104A300008950F931F93CF93DF938C01862F6EEF12
:104A400073E00E94140E892B91F4C091FE03D09163
:104A5000FF03209761F0F8018281833039F4CE01A1
:104A6000DDDFCE01DBDFCE01D9DF01C0E0F7DF9172
:104A7000CF911F910F9108950F931F93CF93DF93C1
:104A80008C01EB016EEF73E08C2F0E94140E892BCA
:104A900009F057C0FE01FF27D80112968C9112979A
:104AA000E05DFD4F8130A9F415968C9182FD4EC0DA
:104AB00080FF4CC082E080838091000490910104CB
:104AC0000097B9F48091FE039091FF030097C9F11C
:104AD00010C08230A1F515968C9182FD26C080FD14
:104AE0000AC083E0808380910204909103040097C0
:104AF000F1F041DF26C084E080838091040490912E
:104B000005040097B1F78091FE039091FF03009791
:104B100001F184DF8091000490910104009749F72E
:104B20008091FE039091FF03E4CF85E08083809124
:104B3000FE039091FF03009721F070DFF1CF86E034
:104B40008083DF91CF911F910F91089581E0808341
:104B5000B9CF8091000490910104B8CF0F931F93B7
:104B6000CF93DF938C01EB016EEF73E08C2F0E94EB
:104B7000140E892B71F4DD27C05DDD4F8881F801AB
:104B8000128218828330E9F048F4813059F0823083
:104B900081F0DF91CF911F910F9108958430B1F092
:104BA0008530B9F78091FE039091FF03009789F358
:104BB00006C08091000490910104009799F3FCDEF7
:104BC000E8CF8091020490910304F7CF8091040410
:104BD00090910504009799F72091FE033091FF030F
:104BE000809100049091010421153105F9F200979C
:104BF00031F7C901E4CFCF93DF93A8E3B1E06EE3CF
:104C000071E041E030E02D912F3F79F0E22FE29505
:104C1000EF70E05EF0E0808190E02F7002C095952B
:104C200087952A95E2F780FF22C080E0382B440F59
:104C30006A177B0741F78091490283131AC080915C
:104C4000C001811509F1C091BE01D091BF010E9440
:104C50001A108C1B9D0B0597B8F08091490290911A
:104C600081038913809381031092C0010DC0842FAA
:104C7000DDCF3093490281E08093C0010E941A1079
:104C80009093BF018093BE01DF91CF910895CDB77E
:104C9000DEB7E0970FB6F894DEBF0FBECDBF85B785
:104CA000806885BF85B7806885BF84B7877F84BFEC
:104CB0000FB6F894A8958091600088618093600099
:104CC000109260000FBE80E890E00FB6F8948093D9
:104CD0006100909361000FBE81E08093030181E445
:104CE00096E09093B5018093B4010E9450060E9413
:104CF000510D0E94950D8AE0E5E1F1E0DE0111968B
:104D000001900D928A95E1F7FE0131969E01255F93
:104D10003F4FEFA7F8AB41E050E08191A82FA2955B
:104D2000AF70B0E091966C9191978F708A0102C03C
:104D3000000F111F8A95E2F7C801962F982B9196C4
:104D40009C93919792969C919297809589239296A5
:104D50008C93E217F30709F70E94DD080E943A09D5
:104D60008091E20084608093E200789480918403D3
:104D7000811599F08091E9001091EC008F701795E2
:104D800011271795182B1092E9008091E80083FDF8
:104D90000E94ED131F701093E90082E084BD93E040
:104DA00095BD9DE797BD80936E000E94C10C811157
:104DB00002C00E947F0EEFE6F3E088E0DF011D9263
:104DC0008A95E9F784988C98809888981092640363
:104DD00010926203109263038FEF93E09093DB02D3
:104DE0008093DA021092D9021092D8021092D70260
:104DF0001092D60210925902109258021092570245
:104E00001092560210926C0310926B039093610300
:104E10008093600310925F0310925E0310925D0313
:104E200010925C031092DF021092DE021092DD02FB
:104E30001092DC0210926A031092690310926803C8
:104E4000109267031092660310926503A8E3B1E025
:104E50002EE331E041E050E08D918F3FA1F0E82F4B
:104E6000E295EF70F0E061A18F708A0102C0000F3F
:104E7000111F8A95E2F7C801902F9095962391A370
:104E800092A1892B82A32A173B0731F71092810345
:104E90001092490280E090E00E944F32833E9E4F84
:104EA00021F40E94C10C81111DC063EE7EEF80E0F1
:104EB00090E00E947D3260E082E090E00E946332E8
:104EC00081E08093CB0561E083E090E00E94633253
:104ED00060E074E184E090E00E947D320E947F0EE9
:104EE0000E94B30982E090E00E94423280934C021B
:104EF00084E090E00E944F329093CE058093CD05E0
:104F00007ADE8FE59AEE0197F1F700C0000073DEBC
:104F10008091810383FF08C06FEF7FEF80E090E016
:104F20000E947D320E94C90983E090E00E944232D3
:104F30000E9497030E94170F8FE090E00E944A3270
:104F40006093CF057093D0058093D1059093D205DF
:104F5000663010F00E94B309E091CF05F0E0EE0F4B
:104F6000FF1FE655FE4F808191810E94070F84E06C
:104F700091E090938C0380938B0382E0282E33245E
:104F8000339480918403853049F480918403853083
:104F900009F434C10E94B3130E941E072CDE8091D5
:104FA0004D02E09081038E11C6C6C3DC00918504DA
:104FB000109186040115110591F1C0905202D09014
:104FC0005302E0905402F09055020E94E6076C19DB
:104FD0007D098E099F09C0904E02D0904F02E0904B
:104FE0005002F09051026C157D058E059F05B8F0BA
:104FF000C8010E94571210928604109285041092E4
:1050000052021092530210925402109255021092C2
:105010004E0210924F021092500210925102E090F4
:105020000D05F0900E05E114F10441F100910F051A
:10503000109110050E941A109C01201B310B890150
:10504000C7010E94290E80179107C0F420910D0519
:1050500030910E05C9019927287F3327232B09F0AA
:1050600019C114E0880F991F1A95E1F783579B4FD8
:10507000DC0115962C9122FF0E94BA10809111013B
:10508000811511F10091C9051091CA05011511058D
:10509000D9F00E941A10801B910B20915C05309171
:1050A0005D052817390780F490915F0580915E05B2
:1050B000981709F4F2C062D910925D0510925C0550
:1050C0001092CA051092C90580917703811551F09D
:1050D00010927703809171038093720380916F0324
:1050E0008093700384EFF8D72C0180EFF5D73C0153
:1050F00080916C03811521F080916B0381112BC08D
:10510000EBE6F3E0FF93EF932CE633E03F932F932E
:10511000E6E58E2EE2E09E2EF8E5AF2EF2E0BF2E01
:10512000AAE5CA2EA2E0DA2EB8E9EB2EB2E0FB2EF9
:1051300006ED12E027ED32E048ED52E06AED72E054
:10514000C2010E945C0290936803809367030F90F2
:105150000F900F900F9080916A03811521F080913C
:10516000690381112BC069E673E07F936F93AAE610
:10517000B3E0BF93AF934CED842E42E0942E5EEDEE
:10518000A52E52E0B52E60EEC62E62E0D62E7EE150
:10519000E72E73E0F72E0CE513E02DE533E04EE546
:1051A00053E060E673E0C3010E945C0290936603E3
:1051B000809365030F900F900F900F9040916703BD
:1051C0005091680380916503909166032091640378
:1051D000211178C04416550608F067C06816790694
:1051E00008F480C083E08093640380916303811599
:1051F00009F478C01092630311E075C080918403B4
:10520000843031F10E94AC0A10924A02A8E1B0E069
:10521000E0E40FB6F894A895A09360000FBEE09369
:10522000600083B7817F846083BF83B7816083BF61
:105230007894889583B78E7F83BF0FB6F894A8952E
:1052400080916000886180936000109260000FBEC2
:10525000D2DC80918103811509F497CE80914B02B5
:10526000811509F492CE19BCF2E0F9BD09B400FE33
:10527000FDCF8091D8008F7D8093D8008091E00091
:1052800082608093E0008091E00081FDFCCF0E946D
:10529000B3137BCE80E090E0EBCE2AD81092CA0503
:1052A0001092C9050E9468060FCF68167906D0F4DF
:1052B00030926403809162038115A1F01092620321
:1052C0001FEF11C0213009F079C04416550608F4CB
:1052D0006EC06816790630F0109264032093630361
:1052E0001092620310E0E090FC03F090FD030E9436
:1052F0001A108E199F0984369105B0F1E0906D0364
:10530000F0906E030E941A108E199F09059760F1A4
:105310008091FB03811128C0111531F18091710337
:1053200090E09C012F5F3F4F237033274091720321
:105330004217130699F081599C4F41E0113009F052
:1053400040E0479544274795DC0114964C93209301
:10535000710380916F038F5F80936F030E941A1017
:1053600090936E0380936D0380E01AED2091720399
:1053700090917103921709F458C030E0F901ED588B
:10538000FC4F808187FB882780F92F5F3F4F237078
:10539000332720937203909170039F5F9093700363
:1053A000B12FB81B8B2F0E94B01281E0DFCF68169F
:1053B000790608F097CF2092640390CF223001F550
:1053C0004416550670F06816790608F08BCF3092B7
:1053D000640380916203811509F484CF1092620303
:1053E0000BCF6816790608F47DCF83E080936403C1
:1053F00080916303811509F475CF1092630360CF28
:105400004416550658F06816790608F46BCF1092CA
:105410006403309262031092630364CF68167906C6
:1054200008F060CF20926403F4CF81110E94E60758
:105430000E94AC0A81110E94E60786E0EEEEF3E0DE
:10544000AFA5B8A901900D928A95E1F71092F003EB
:105450001092F1031092F2031092F3038B819C815E
:10546000892B811509F443C000917A0310917B03C5
:105470000E941A109C01201B310B9091EC03911596
:1054800009F454C42531310590F19F3F19F09F5F15
:105490009093EC031B81111559F00E94D40691E002
:1054A00011160CF09FEF899F802D11248093F0033B
:1054B0001C81111559F00E94D40691E011160CF0D0
:1054C0009FEF899F802D11248093F1038091F00339
:1054D000811569F01091F103111549F00E94C6067B
:1054E0008093F003812F0E94C6068093F1038D8183
:1054F0009E81892B811509F443C000917803109196
:1055000079030E941A109C01201B310B9091EB0330
:10551000911509F406C42135310590F19F3F19F02A
:105520009F5F9093EB031D81111559F00E94F406C3
:1055300091E011160CF09FEF899F802D112480932C
:10554000F2031E81111559F00E94F40691E0111624
:105550000CF09FEF899F802D11248093F30380919D
:10556000F203811569F01091F303111549F00E94BF
:10557000C6068093F203812F0E94C6068093F30330
:105580006FA578A98EEE93E00E94B60781110CC03A
:105590008091F0039091F103892B9091F203892B74
:1055A0009091F303892B81110E940D1186E0EFA5E4
:1055B000F8A9AEEEB3E001900D928A95E1F70E9452
:1055C0001E0790917C03891721F080937C030E9431
:1055D000E60780918403843009F0D3CC83E0809384
:1055E000E9008091E80082FFCCCC8091E80090E057
:1055F00085FF05C00E94AC08811519F191E08091EA
:10560000E8008B778093E800911509F4BACC0091FB
:10561000870310918803E9810115110571F1EE3FAF
:1056200009F04DC08A81833020F08550833008F026
:1056300046C0EA81EE3008F042C0F0E0ED58FB4C85
:10564000E7C600E210E0FE0131967F018091E8009C
:1056500085FD0AC08091E8008B778093E8000E9466
:10566000AC08811599F3CACF8091F100D7018D93D1
:105670007D010150104051F7C1CFE43148F4E115EC
:1056800049F0E150E33130F4F0E0EF57FB4CC0C695
:10569000EE3F79F28FEF898312C01A8289E08B8303
:1056A0000EC08A81823081F08330B1F0813091F771
:1056B0000E94E607B3D66B837C838D839E83CE01E5
:1056C00001960E94FC085DCC88E290E0DBD61B824C
:1056D0001C821D828E83F3CF80918203909183037D
:1056E000892B69F380918103DACF8A81823091F628
:1056F0006B817C818D819E8191D688E290E0E3D69A
:10570000DECF4C816B818A810E94E30B9827892729
:1057100098279E838D83D3CF2D813E8132272327E7
:1057200032274C816B818A810E94650AC8CF0E9412
:10573000DA0CC5CF80E18A83C2CF82E08A8387EA10
:10574000AECF8C818D3108F0BACF8A809B809824AF
:1057500089249824A12CB12C8E010F5F1F4F780152
:10576000E80EF11C0E151F0509F4A9CF80E0B7EA79
:105770008B16B2E09B06A104B10420F4C401875A41
:105780009E4F80D6F80184830F5F1F4FFFEF8F1A63
:105790009F0AAF0ABF0AE6CF8091820390918303EC
:1057A000892B09F48CCF8C818D3108F088CF882E1D
:1057B000912CA12CB12CCA80DB80DC24CD24DC24EC
:1057C000E12CF12C8E010F5F1F4F412C512C320127
:1057D000481459046A047B0408F071CF27EAC21602
:1057E00022E0D206E104F10438F4D80114966C9159
:1057F000C601875A9E4F67D6BFEF4B1A5B0A6B0AEA
:105800007B0AEFEFCE1ADE0AEE0AFE0A0F5F1F4F89
:10581000DFCF0E94440E53CF84E08DCF8C818D3139
:1058200008F04DCF882E912CA12CB12CCA80DB80A2
:10583000DC24CD24DC24E12CF12C412C512C320130
:105840008E010B5F1F4F481459046A047B0408F053
:1058500036CF80E0F0E3CF16D104E104F10418F470
:10586000C60189960FD6D8018D938D01BFEF4B1AD3
:105870005B0A6B0A7B0AEFEFCE1ADE0AEE0AFE0A1B
:10588000E2CF2C81622E712C2D3108F018CF8A8145
:105890009B819827892798274C01A12CB12C803314
:1058A000910508F00CCF422F50E060E070E04BA76C
:1058B0005CA76DA77EA740E350E060E070E0481968
:1058C00059096A097B09421751056105710508F4F8
:1058D000F6CE2091820330918303232B09F03EC042
:1058E0007C0159E2E50EF11C80FBCC24DD24C0F8DC
:1058F00080FF0BC08896C6D59D8189279827892768
:1059000081159C4711F48FEF8D838BA59CA5ADA5C8
:10591000BEA5880D991DAA1DBB1D80FF17C0830160
:105920000150110935E0432E512C4C0E5D1E400EE6
:10593000511EC701860D971DA5D5D2019C918115D9
:105940009C4719F48FEFF20180833801FE013196F4
:10595000EC0DFD1D2FEFC614D70438F08E010F5F3C
:105960001F4FC12CD12C760124C0948185818115D3
:105970009C4711F42483258312E0C10ED11C32967A
:10598000EACF20E382169104A104B10430F4D801D7
:1059900014966C91C401899696D5BFEFCB1ADB0A99
:1059A000EB0AFB0AEFEF8E1A9E0AAE0ABE0A0F5FE1
:1059B0001F4F2BA53CA54DA55EA5C216D306E40638
:1059C000F506F8F27CCE8091820390918303892BB7
:1059D00009F475CECE0101960E94FC083FEF40E726
:1059E00052E0315040405040E1F700C000009ACAF8
:1059F00088E0E0E2F1E0DE01919601900D928A9557
:105A0000E1F7FE0132968FE1DF011D928A95E9F7F9
:105A100086E0898388E07F96DE01159601900D92DD
:105A20008A95E1F74CCE8CE3898381E08A831B82DF
:105A30001C8245CE8B819C81092E000CAA0BBB0BCE
:105A400025E0880F991FAA1FBB1F2A95D1F7AC012B
:105A5000BD01405E5F4F6F4F7F4F481759076A0780
:105A60007B0708F42CCE8C33E1E09E07A105B1053D
:105A700008F025CE4D33F1E05F076105710520F098
:105A80004CE351E060E070E0481B590BBC01665FDD
:105A90007C4FCE010196C9D412CE4AE150E06FEF9F
:105AA00070E0CE010796D7D48091820389830A8360
:105AB0001B8283E08C831D8285E00CCE81E090E028
:105AC000909388038093870382E390E09093800310
:105AD00080937F030E941A1090937E0380937D032E
:105AE000EECD0115110571F1D0908103E0907D0399
:105AF000F0907E030E941A108E199F098536910539
:105B000040F1D5FE26C0D3FE24C00E941A10909307
:105B10007E0380937D0380917F03909180030197A2
:105B20009093800380937F03892B61F41092880304
:105B30001092870381E090E0909383038093820327
:105B400000E010E08091820389830A8380917F03C3
:105B5000A6CD82E390E09093800380937F03F2CF01
:105B60001092830310928203AACD40E250E06FEFBF
:105B700070E0CE0101966FD4A2CDEB81E73008F042
:105B80009ECDF0E0EC56FB4C43C4FE0134968DE113
:105B9000DF011D928A95E9F788E089838A837FCDAA
:105BA0008C819AE0F92E8E010F5D1F4FF8012F2D89
:105BB00011922A95E9F7B8010E94140E8983F80121
:105BC000DE01129601900D92FA94E1F778CD1C81D6
:105BD0008AE0FE013596DE01919601900D928A953C
:105BE000E1F789A19AA10E9443069AA389A38BA1F8
:105BF0009CA10E9443069CA38BA38DA19EA10E9401
:105C000043069EA38DA38FA198A50E94430698A743
:105C10008FA38FEF183060F43AE0139FB001112486
:105C200067597F4F4AE050E0CE0181966AD480E008
:105C300089830E94500643CD2C816AE0CE01819673
:105C4000DC01E62F1D92EA95E9F7283008F044C000
:105C5000629FB001112467547F4F4AE050E002D4A4
:105C600080E089838AE0FE01B196DE011296D6CEED
:105C70001C818AE0FE013596DE01919601900D921D
:105C80008A95E1F789A59AA50E9443069AA789A754
:105C90008FEF183060F4FAE01F9FB00111246754B1
:105CA0007F4F4AE050E0CE0181962BD480E089837B
:105CB0000E94510D04CD2C816AE0CE018196DC0159
:105CC000E62F1D92EA95E9F7283030F4629FB00183
:105CD0001124675F7E4FC1CF8FEFC3CF1C818AE055
:105CE000FE013596DE01919601900D928A95E1F7BD
:105CF0008BA19CA10E9443069CA38BA38FEF18301D
:105D000060F4FAE01F9FB0011124675F7E4F4AE004
:105D100050E0CE018196F5D380E089830E94950DF5
:105D2000CECC2B30310508F0FBCB2ACC2B30310503
:105D300008F0ADCBDCCBF82EFE2400E011E08F2D77
:105D400081238115A9F009831A820E941A109C836D
:105D50008B833D8291E08E2D8123811101C090E0E3
:105D60009E8349815A816B817C818D810E946B2247
:105D70000F5F110F063019F7E0924D020E94E607FF
:105D800015C978941F921FB61F9211248F939F9369
:105D9000AF93BF938091D6019091D701A091D80184
:105DA000B091D9010196A11DB11D8093D6019093A8
:105DB000D701A093D801B093D901BF91AF919F9122
:105DC0008F911F901FBE1F9018951F920F920FB6B4
:105DD0000F9211242F933F934F935F936F937F9371
:105DE0008F939F93AF93BF93EF93FF938091E100C5
:105DF00082FF09C08091E20082FF05C08091E1002E
:105E00008B7F8093E1008091DA0080FF23C0809136
:105E1000D80080FF1FC08091DA008E7F8093DA0067
:105E20008091D90019BC80FFA6C082E089BD09B469
:105E300000FEFDCF81E0809384038091C501811134
:105E400009C00E94DD080E943A098091E200846046
:105E50008093E2008091E10080FF1AC08091E2000F
:105E600080FF16C08091E2008E7F8093E2008091D7
:105E7000E20080618093E2008091D800806280938C
:105E8000D80019BC85E08093840383E080930301EC
:105E90008091E10084FF2EC08091E20084FF2AC03F
:105EA00019BC82E089BD09B400FEFDCF8091D80005
:105EB0008F7D8093D8008091E1008F7E8093E100F8
:105EC0008091E2008F7E8093E2008091E200816009
:105ED0008093E2008091C401811509F451C084E0EF
:105EE0008093840380918403843009F051C082E060
:105EF000809303018091E10083FF2CC08091E20038
:105F000083FF28C08091E100877F8093E10082E0D9
:105F1000809384031092C4018091E1008E7F80936E
:105F2000E1008091E2008E7F8093E2008091E200A8
:105F300080618093E20042E060E080E00E940A0914
:105F40008091F00088608093F00081E080930301ED
:105F500080930201FF91EF91BF91AF919F918F913B
:105F60007F916F915F914F913F912F910F900FBE55
:105F70000F901F901895109284031092C5016ACF5C
:105F80008091E30087FF02C083E0AACF81E0A8CF21
:105F900081E0AECF1F920F920FB60F921124EF92B5
:105FA000FF920F931F932F933F934F935F936F93A2
:105FB0007F938F939F93AF93BF93CF93EF93FF9371
:105FC00009EE10E0F8018081C091EC008F70C79558
:105FD000CC27C795C82B108280EFE82EF12CF70153
:105FE0008081877F808378940E94ED13F80110826E
:105FF000F701808188608083CF70F801C083FF91B2
:10600000EF91CF91BF91AF919F918F917F916F91C0
:106010005F914F913F912F911F910F91FF90EF90C2
:106020000F900FBE0F901F901895803F09F188F4D4
:10603000843901F140F48533F9F08633F9F0843383
:1060400039F583E208958639D9F0873909F582E276
:106050000895853FB9F030F4813FB1F0843FC1F439
:1060600084E00895863F91F0873F91F487E008959A
:1060700080E0089580E2089584E2089585E208951D
:1060800081E2089585E0089581E0089586E008950D
:106090008FE1089595E890937A00982F9072906818
:1060A00090937B008F7190911201892B80937C00DB
:1060B00080917A00806480937A0080917A0086FDD6
:1060C000FCCF809178002091790090917A009F77A1
:1060D00090937A00922F0895A8DFDCCF289A219A16
:1060E000229A23982B9880E58CBD0895FC0180911D
:1060F00014018F3F09F085C080818F3F09F481C072
:106100001092D4058181811519F080E28093D40525
:1061100092818091D405923009F44FC0933009F4F4
:1061200050C08460913009F449C08381948121E09A
:1061300030E02817390708F446C08091D405203292
:10614000310509F456C008F041C02830310509F482
:106150004BC02031310509F44AC02230310509F421
:106160003FC08CB59091D405892B8CBD8091D3050F
:10617000811519F08DB581608DBD208120931401AA
:10618000458140931301E22FE295EF70A1E2AE0F3B
:10619000B0E03C912F7081E090E001C0880F2A951B
:1061A000EAF7232F282B2C93EE5DF0E0908141112C
:1061B00025C0892B808381E0089588608093D40571
:1061C000B4CF8C60FBCF220F331FB3CF2034310507
:1061D00099F083602038310521F68093D405C1CF32
:1061E00081E08093D305BDCF91E09093D30581608A
:1061F000F4CF91E09093D3058260EFCF809589230F
:10620000D9CF80E00895A6E0B0E0E8E0F1E3B2C0C5
:1062100089836A834B833D832C8381E08E83CE0107
:10622000019664DF2696E2E0C1C0CF93DF938EBD76
:106230000E941A10EC010DB407FE05C08EB590E067
:10624000DF91CF9108950E941A108C1B9D0B84360C
:10625000910588F38EEF9FEFF3CFCF93DF931EBCB2
:106260000E941A10EC010DB407FE05C08EB590E037
:10627000DF91CF9108950E941A108C1B9D0B8436DC
:10628000910588F38EEF9FEFF3CF0F931F93CF937A
:10629000DF93EC018C01060F171FC017D10739F4EB
:1062A00080E090E0DF91CF911F910F910895899147
:1062B000BCDF97FFF2CF8EEF9FEFF4CF0F931F93CA
:1062C000CF93DF93EC018C01060F171FC017D10786
:1062D00039F480E090E0DF91CF911F910F91089504
:1062E000BCDF97FD02C08993F1CF8EEF9FEFF3CF14
:1062F000209114012F3F51F1E22FE295EF70A1E2BE
:10630000AE0FB0E03C912F7081E090E001C0880FAB
:106310002A95EAF7232F282B2C93EE5DF0E02091AD
:1063200013019081211599F0892B80838FEF809341
:1063300014018DB58E7F8DBD9CB58091D40580955F
:1063400089238CBD1092D4051092D30508958095B1
:106350008923EBCF2F923F924F925F926F927F9261
:106360008F929F92AF92BF92CF92DF92EF92FF9265
:106370000F931F93CF93DF93CDB7DEB7CA1BDB0B11
:106380000FB6F894DEBF0FBECDBF09942A883988B6
:1063900048885F846E847D848C849B84AA84B984BD
:1063A000C884DF80EE80FD800C811B81AA81B981C9
:1063B000CE0FD11D0FB6F894DEBF0FBECDBFED01DD
:1063C0000895AA1BBB1B51E107C0AA1FBB1FA6173C
:1063D000B70710F0A61BB70B881F991F5A95A9F78E
:1063E00080959095BC01CD01089597FB072E16F47A
:1063F000009406D077FD08D0E4DF07FC05D03EF41A
:10640000909581959F4F0895709561957F4F089560
:10641000EE0FFF1F0590F491E02D09946927962750
:1064200069277827872778270895FB01DC0102C0B8
:1064300005900D9241505040D8F70895FB01DC01C2
:1064400004C08D910190801921F441505040C8F74B
:10645000881B990B0895DC0101C06D934150504099
:10646000E0F70895DC01CB01FC01F999FECF06C0ED
:10647000F2BDE1BDF89A319600B40D924150504002
:10648000B8F70895F999FECF92BD81BDF89A992782
:1064900080B50895A6E1B0E044E050E0E5CFA8E182
:1064A000B0E042E050E0E0CFDC01A40FB51F415066
:1064B000504040F0CB01840F951F2E9105D04150E4
:1064C0005040D8F70895262FF999FECF92BD81BD8F
:1064D000F89A019700B4021639F01FBA20BD0FB622
:1064E000F894FA9AF99A0FBE08950396272FECDFD5
:1064F000EADF252FE9DF242FE7CF0196272FE4DFFE
:10650000E2CFDC01CB0102C02D9105D041505040BB
:10651000D8F70895262FF999FECF1FBA92BD81BDF5
:1065200020BD0FB6F894FA9AF99A0FBE0196089515
:106530005058BB27AA270ED0E5C0D6D030F0DBD00C
:1065400020F031F49F3F11F41EF4CBC00EF4E0951F
:10655000E7FBC1C0E92FE7D080F3BA1762077307E2
:106560008407950718F071F49EF5FFC00EF4E095CE
:106570000B2EBA2FA02D0B01B90190010C01CA01FD
:10658000A0011124FF27591B99F0593F50F4503EA8
:1065900068F11A16F040A22F232F342F4427585F9A
:1065A000F3CF469537952795A795F0405395C9F7B2
:1065B0007EF41F16BA0B620B730B840BBAF091506A
:1065C000A1F0FF0FBB1F661F771F881FC2F70EC009
:1065D000BA0F621F731F841F48F4879577956795DC
:1065E000B795F7959E3F08F0B3CF9395880F08F0C5
:1065F0009927EE0F97958795089504D06894B11167
:10660000B5C0089598D088F09F5790F0B92F99277A
:10661000B751A0F0D1F0660F771F881F991F1AF0AD
:10662000BA95C9F712C0B13081F09FD0B1E008959A
:106630009CC0672F782F8827B85F39F0B93FCCF31B
:10664000869577956795B395D9F73EF490958095A3
:10665000709561957F4F8F4F9F4F0895E89409C0C3
:1066600097FB3EF490958095709561957F4F8F4F85
:106670009F4F9923A9F0F92F96E9BB279395F6959B
:10668000879577956795B795F111F8CFFAF4BB0F19
:1066900011F460FF1BC06F5F7F4F8F4F9F4F16C07D
:1066A000882311F096E911C0772321F09EE8872F07
:1066B000762F05C0662371F096E8862F70E060E0C3
:1066C0002AF09A95660F771F881FDAF7880F96953C
:1066D000879597F9089597F99F6780E870E060E0E3
:1066E00008959FEF80EC089500240A94161617066B
:1066F00018060906089500240A94121613061406B3
:1067000005060895092E0394000C11F4882352F015
:10671000BB0F40F4BF2B11F460FF04C06F5F7F4FCD
:106720008F4F9F4F089557FD9058440F551F59F0B4
:106730005F3F71F04795880F97FB991F61F09F3F6E
:1067400079F087950895121613061406551FF2CF97
:106750004695F1DF08C0161617061806991FF1CFE7
:1067600086957105610508940895E894BB2766270E
:106770007727CB0197F908950BD0C4CFB5DF28F068
:10678000BADF18F0952309F0A6CFABCF1124EECFD6
:10679000CADFA0F3959FD1F3950F50E0551F629F7C
:1067A000F001729FBB27F00DB11D639FAA27F00D6A
:1067B000B11DAA1F649F6627B00DA11D661F829F91
:1067C0002227B00DA11D621F739FB00DA11D621F76
:1067D000839FA00D611D221F749F3327A00D611D93
:1067E000231F849F600D211D822F762F6A2F112475
:1067F0009F5750408AF0E1F088234AF0EE0FFF1FC8
:10680000BB1F661F771F881F91505040A9F79E3FFE
:10681000510570F060CFAACF5F3FECF3983EDCF3F8
:10682000869577956795B795F795E7959F5FC1F73B
:10683000FE2B880F911D9695879597F90895F894EA
:10684000FFCF34113A113D1143115811581158110D
:106850005811581158115811581146114B114F1118
:1068600055117A1180118411CE14F414FA14F41411
:10687000FA144D156F15FA1476168316961BFE1B27
:106880009E1B691B6D1BA21B711BA61BB21B7D1BD4
:10689000F71B811BB61B851BBA1BDF1B891BBE1B8D
:1068A000E61B8E1BC41BCC1B751BAA1B791BAE1BC6
:1068B000921BC81BD61BEF1BF51B631B9A1B051CE9
:1068C000361B3C1B291B301B421B481B4E1BDE1C6E
:1068D000DE1C171D171DC91DE41D3D1D3D1DE91DB5
:1068E0005C1E6D1E6D1EF82C132D1A2D5F2B5F2B59
:1068F0004D2D5E2D712DB02DB52D5F2B5F2B5F2B98
:10690000BD2D4D2B512B752B812B8C2B972B4A2B6F
:106910004A2B4A2B4A2BE32C9A2B9D2BA12BCC2BB9
:10692000092C0C2C0E2C412CC52DD02DE72D1C2E06
:06693000382E5B2E6E2ED6
:1069360000000100E3072F0A3308450A4A0A260A1F
:1069460001014001FF919334379667F6F5F3F7009E
:10695600D16AE92AC4D016350044227B49012701B1
:10696600AC004F026802880295369492C697E20000
:10697600E900EA00B500B600B700CD008301CC00FF
:106986008A01920194012102230224022502260291
:1069960027022A02B300B4006F0070009F01CB01EA
:1069A6009F02A002E200E900EA00B500B600B700C7
:1069B600CD008301CC008A019201940121022302B9
:1069C60024022502260227022A02B300B4006F0021
:1069D60070009F01CB019F02A00258028403B004FD
:0469E60040066009FE
:00000001FF
